:100000000C9450070C9475070C9475070C947507A5
:100010000C9475070C9475070C9475070C94750770
:100020000C9475070C9475070C94EE470C940A48D1
:100030000C9475070C9475070C9475070C94750750
:100040000C9475070C9475070C9475070C94750740
:100050000C9475070C9475070C9475070C94750730
:100060000C9475070C9475070C9475070C94750720
:100070000C9475070C9475070C9475070C94750710
:100080000C9475070C9475070C9475070C94750700
:100090000C9475070C9475070C9475070C94FD4926
:1000A0000C943A4A0C94774A0C94B44A0C94750711
:1000B0000C9475070C9475070C9475070C947507D0
:1000C0000C9475070C9475070C9475070C947507C0
:1000D0000C9475070C9475070C9475070C947507B0
:1000E0000C9475070C9475070C9475070C947507A0
:1000F0000C9475070C9475070C9475070C94750790
:100100000C9475070C9475070C9475070C9475077F
:100110000C9475070C9475070C9475070C94094999
:100120000C9446490C9483490C94C0490C9475076F
:100130000C9475070C9475070C9475070C9475074F
:100140000C9475070C9475070C9475070C9475073F
:100150000C9475070C9475070C9475070C9475072F
:100160000C9475070C9475070C9475070C9475071F
:100170000C9475070C9475070C9475070C9475070F
:100180000C9475070C9475070C9475070C947507FF
:100190000C9475070C9475070C9475070C947507EF
:1001A0000C9475070C9475070C9475070C947507DF
:1001B0000C9475070C9475070C9475070C947507CF
:1001C0000C9475070C9475070C9475070C947507BF
:1001D0000C9475070C9475070C9475070C947507AF
:1001E0000C9475070C9475070C9475070C9475079F
:1001F0000C9475073C696E70757420747970653D58
:10020000227375626D697422207374796C653D2266
:100210006865696768743A203530707822206E61AD
:100220006D653D22746F67676C65222076616C7521
:10023000653D224C454434223E266E627370266E24
:100240006273703C696E70757420747970653D22BC
:100250007375626D697422207374796C653D2268D0
:1002600065696768743A203530707822206E616D58
:10027000653D22746F67676C65222076616C7565D9
:100280003D224C454435223E266E627370266E62D6
:1002900073703C696E70757420747970653D22735B
:1002A00075626D697422207374796C653D2268658E
:1002B000696768743A203530707822206E616D6508
:1002C0003D22746F67676C65222076616C75653DB1
:1002D000224C454436223E266E627370266E62734F
:1002E000703C696E70757420747970653D22737509
:1002F000626D697422207374796C653D226865694A
:100300006768743A203530707822206E616D653DE3
:1003100022746F67676C65222076616C75653D227B
:100320004C454437223E266E627370266E627370AF
:100330003C2F6669656C647365743E3C2F666F7212
:100340006D3E3C2F74643E3C74643E266E62737056
:100350003B3C2F74643E3C2F74723E3C2F746162B0
:100360006C653E3C2F74643E3C7464207769647411
:10037000683D22323025223E3C2F74643E3C2F746F
:10038000723E3C2F7461626C653E3C2F626F6479F3
:100390003E3C2F68746D6C3E003C74723E3C74644D
:1003A0003E3C666F726D206D6574686F643D2267B8
:1003B00065742220616374696F6E3D22223E3C7039
:1003C0003E3C696E70757420747970653D2273755A
:1003D000626D697422207374796C653D2268656969
:1003E0006768743A2035307078222076616C7565C4
:1003F0003D2252656672657368223E3C2F703E3C1A
:100400002F666F726D3E3C2F74643E3C2F74723EBB
:100410003C2F7461626C653E3C62723E3C666F725A
:100420006D2069643D22666F726D226E616D653D5F
:1004300022666F726D22206D6574686F643D22675D
:1004400065742220616374696F6E3D22696E646514
:10045000782E68746D6C223E3C6669656C647365C9
:10046000743E3C6C6567656E643E4C454420636F2A
:100470006E74726F6C3C2F6C6567656E643E3C6990
:100480006E70757420747970653D227375626D6944
:100490007422207374796C653D226865696768749D
:1004A0003A203530707822206E616D653D22746F80
:1004B00067676C65222076616C75653D224C45440A
:1004C00030223E266E627370266E6273703C696ED7
:1004D00070757420747970653D227375626D6974EE
:1004E00022207374796C653D226865696768743A87
:1004F000203530707822206E616D653D22746F6703
:10050000676C65222076616C75653D224C454431EF
:10051000223E266E627370266E6273703C696E7046
:10052000757420747970653D227375626D697422EB
:10053000207374796C653D226865696768743A2038
:100540003530707822206E616D653D22746F67676B
:100550006C65222076616C75653D224C45443222E3
:100560003E266E627370266E6273703C696E7075A3
:100570007420747970653D227375626D69742220F0
:100580007374796C653D226865696768743A2035D3
:1005900030707822206E616D653D22746F67676CE4
:1005A00065222076616C75653D224C454433223EC0
:1005B000266E627370266E6273703C703E003C2F34
:1005C00074643E3C74643E3C623E3C2F623E3C2F71
:1005D00074643E3C2F74723E003C74723E3C746402
:1005E0003E4D414320416464726573733A20003C80
:1005F0002F74643E3C74643E3C623E3C2F623E3C41
:100600002F74643E3C2F74723E003C74723E3C7406
:10061000643E495020416464726573733A20004817
:100620005454502F312E3020323030204F4B0A534B
:1006300065727665723A20776C705F687474706466
:100640000A436F6E74656E742D747970653A207408
:100650006578742F68746D6C0A0A3C21444F4354CA
:100660005950452048544D4C205055424C49432048
:10067000222D2F2F5733432F2F4454442048544DBD
:100680004C20342E3031205472616E736974696F5E
:100690006E616C2F2F454E222022687474703A2FA1
:1006A0002F7777772E77332E6F72672F54522F68FC
:1006B000746D6C342F6C6F6F73652E647464223E9E
:1006C0003C68746D6C3E3C686561643E3C74697462
:1006D0006C653E6F574C207069636F2048545450CE
:1006E00020576562207365727665723C2F74697459
:1006F0006C653E3C2F686561643E3C626F647920A6
:100700007374796C653D666F6E742D66616D696C8E
:10071000793A617269616C3E3C7461626C653E3C21
:1007200074723E3C74642077696474683D22313091
:1007300030223E3C2F74643E3C74643E3C746162E3
:100740006C653E3C74722076616C69676E3D227404
:100750006F70223E3C74643E3C696D672073726327
:100760003D226C6F676F2E6769662220616C743D55
:10077000226C6F676F227469746C653D226C6F67C1
:100780006F223E3C2F74643E3C2F74723E3C747268
:100790003E3C74642077696474683D2235303022B1
:1007A0003E3C68323E576562205365727665722022
:1007B00072756E6E696E67206F6E206F574C207079
:1007C00069636F3C2F68323E3C703E546865207709
:1007D0006562207061676520697320736572766554
:1007E0006420627920776C705F687474706420751F
:1007F00073696E672074686520535042383030202A
:10080000574C414E206D6F64756C6520616E64209D
:10081000746865206F574C2D7069636F26636F7025
:10082000793B20536F667477617265204150493B74
:10083000206120756E697175652057692D466920A4
:10084000736F6C7574696F6E2066726F6D203C6299
:100850003E4826616D703B4420576972656C657334
:10086000732041423C2F623E2E3C2F703E3C68720A
:100870003E3C7461626C653E0047494638396145CB
:10088000017B00A10000FFFFFF006699000000FF50
:10089000FFFF21FE114372656174656420776974FE
:1008A000682047494D50002C0000000045017B00A6
:1008B0000002FE848FA9CBED0FA39CB4DA8BB3DECC
:1008C000BCFB0F86E24896E689A6EACAB6EE0BC7DD
:1008D000F24CD7F68DE7FACEF7FE0F0C0A87C4A2CA
:1008E000F1884C2A97CCA6F3098D4AA7D4AAF58A99
:1008F0006505B6DCAEF70B0E8BC76471F60C2DAB3D
:10090000D7EC36190D3FBAE7F4FA3B8EFFD9F77CE6
:100910007BFE9FD32738C80668384398A81876D836
:10092000D8B2081919E048792279A958A92982D999
:1009300029B809DAE139CA176A8A419A4A77CA3A64
:10094000A1FAEAD62AEB005BAB368BAB60BB6B96A9
:10095000EB0BC01BECF5EB2B6CBC458C7B6C9C3C17
:10096000BB2CDC2CFB1C1CDD3ACD5BCD7ABD9B7D0A
:10097000BA6DDB6DFA5D1B1E3A0E5B0E7AFE9ABEF7
:10098000B9AEDAAEF99E1A5F394F5A4F793F9AEFF6
:10099000B8EFD9AFD1BF4E010F0DC454D0D0C14B69
:1009A00009012D94D4F0CFC34811F34C845411CFD6
:1009B0001DFE5D601A8CF158A6421B04024A9A146F
:1009C000B0E0E4C9942A511E68290366B88D09185D
:1009D00031B0F980A6AB5B2465F6F4F9122800A1CA
:1009E0002D8836D3790027C761123E5EE01954A5E1
:1009F000829625A70A35BA022B31A40694D664DA6A
:100A0000B4D7539D5413503569F6AAD4185A7F7140
:100A100005D6F126D8B07151398DBAF26759BD6843
:100A2000F9BA84D1B6D8DDAF5F4072913B6969E114
:100A30000C64D59E4DBB7647E05C6FBD22987B1958
:100A40009962CC490FD3128BB7AF81B355FDFA9899
:100A5000AC6C70E6C50B58AFDECCB96B6CD996F7B1
:100A60000E255DFA76E4D07F47FBCCCB127883C9A4
:100A7000A879E77EF0B847E5BAB05B2726CC7C754D
:100A800017C4D17503C79DDB366FC82B8962EFCDC4
:100A9000FD7878ED56B10FFFCEE3ADC8D9CE414B0E
:100AA000F7DCDEB5EFC8E8E70BB72FBE2CD0EFF7C9
:100AB000FEF183F78F5B70FC95376020AAD9C5DE05
:100AC0007BD5D1361D75B1FD661E8004E6572080AA
:100AD000018E2760851692365E8438A847C182D081
:100AE000B9D7197B245A87964C2AEEB69D5FDAF166
:100AF000C7228AFFC1789F63C2D9289A0D20EE04CD
:100B00005F4E21C5D7E3880D7628A37F32FE57A418
:100B10008B10C6481E8EE21D69DA04C5DDB0235D68
:100B2000CF41009F8822C2B5A07E6BC1449E914AEE
:100B3000228995931866D85B98E7C5E84395110418
:100B400089E0950ACA39A7661DDAA6618BC62179A4
:100B5000248C51EE59619E63F6F7E1810C0EB914B5
:100B600007B36D79629F377A78E69E0CD0B81F8BF9
:100B700094EE46239A1CEAB09C7C9921C6239D875B
:100B8000DA091B9C1BE658DF84E0A9792AA44E668B
:100B90003A289BB016DAA8659D01F926A2733A3867
:100BA0005BAA8EE6F8A784935E8AAAA5C43EF9FEE6
:100BB0002BA1C9024B43A7268AEAA990BC1A262278
:100BC000A4AD0E5BA356AC3A60A6079B22F76D0D51
:100BD000CEEAFA2990A46E469D8FB69EAA2A9B491A
:100BE0001AB7A6B2DC1AEB6E0653BEABA3A15C3EED
:100BF0006B188F1BE8FB6BBBCCEA29ACA6AB762B42
:100C0000A98B146CABAA81B5322A2A63115BB9E5B2
:100C10008583C64B61BDCB7AC724B109EB991CC152
:100C2000E2EABB2E971E984A71C521DFC927BE5044
:100C3000622C28C794B21CAEC7B4AE5B32B916E8BA
:100C40009CAB7AE18E093391F3FAD9B0C02BB7FA95
:100C5000AAC554920C31CAEDBD37D68FD8BAFB73F2
:100C6000B02F83AB74A4460F0C28D5828EFC70B4D1
:100C7000A34EBC6F8309960AF0D59A0E0D2CC3457E
:100C8000B38DACD0111C0D73CBF95E94484671E066
:100C90009D89DE68F09DB7DF67004E88E08313FE14
:100CA00089E158209EB8E25630DE87E35740AD5EBA
:100CB0008AE45550BE87E597635E87E65470DEB9D7
:100CC000E75280BE8AE851903E87E9A7A33E92EAA8
:100CD0004FB0DEBAEB4DC05E88ECB3D30E95ED4A53
:100CE000E09EBBEE48F02EB5EFBF039FB6F040107C
:100CF0005FBCF16D225FB2F27A30BFA5F3CB437FC8
:100D0000B6F43B505FBDF59C62EFB4F6CA714FB6C6
:100D1000F7D7832F3E11E4976F3EF6E8A74FFDFA11
:100D2000EC23EF7E11CCC72F3FF1F41B01FCFDC378
:100D3000B3AE7F12A4F77F3BC601F0730719A00181
:100D40000F88C0042A70810C6CA0031F08C1084AD8
:100D5000708214ACA0052F8841CD1500003B48548B
:100D600054502F312E3020323030204F4B0A5365F3
:100D7000727665723A20776C705F68747470640A7A
:100D8000436F6E74656E742D747970653A20696D69
:100D90006167652F6769660A0A00485454502F310D
:100DA0002E30203430342046696C65206E6F7420FC
:100DB000666F756E640A5365727665723A20776C59
:100DC000705F68747470640A436F6E74656E742D1E
:100DD000747970653A20746578742F68746D6C0A44
:100DE0000A3C68746D6C3E3C686561643E3C7469A5
:100DF000746C653E6F574C207069636F2048545483
:100E00005020576562207365727665723C2F746955
:100E1000746C653E3C2F686561643E3C626F64792A
:100E20003E3C68323E343034202D205061676520CE
:100E30006E6F7420666F756E643C2F68323E3C7036
:100E40003E536F7272792C207468652070616765FB
:100E500020796F7520617265207265717565737494
:100E6000696E6720776173206E6F7420666F756E90
:100E700064206F6E20746869732073657276657282
:100E80002E3C2F703E3C2F626F64793E3C2F68747D
:100E90006D6C3E006364696E6F70737578585B00AB
:100EA00011241FBECFEFDFE3DEBFCDBF00E00CBFDC
:100EB00018BE19BE1ABE1BBE11E3A0E0B0E2EEE000
:100EC000F7EB00E00BBF02C007900D92A036B10710
:100ED000D9F712E3A0E6B1E301C01D92A33CB1072C
:100EE000E1F70E948A420C94855B0C9400009BB74A
:100EF0008BBFFB018091CA014093CA017DE97093C9
:100F00003400E8958093CA019BBF08952091CF01DA
:100F100027FDFCCF9BB78BBFFB018091CA0123E269
:100F20002093CA010A01E89511248093CA019BBF4E
:100F30000895E0916231F091633108C020813181E0
:100F40002817390729F00380F481E02D3097B1F795
:100F5000CF0108959C01AB01A0916031B091613146
:100F6000ED91FC91119716968D919C911797B9016F
:100F7000199508959C01AB01A0916031B091613148
:100F80001296ED91FC91139716968D919C9117975F
:100F9000B90119950895A0916031B091613114960D
:100FA000ED91FC911597309739F016968D919C91A3
:100FB000179761E070E019950895A0916031B091A4
:100FC00061311496ED91FC911597309739F0169692
:100FD0008D919C91179760E070E019950895E091CC
:100FE0006031F0916131808983FD0CC008951C96B9
:100FF000ED91FC911D97309749F01E968D919C9133
:101000001F971995A0916031B091613151968C91E3
:101010005197882361F351961C9251970895AF928E
:10102000BF92CF92DF92EF92FF920F931F93CF93D5
:10103000DF93EC015B016A01790188E090E0C80E62
:10104000D91EE80EF91EC6010E94F9138883998300
:101050001A82AB821C821D821E820115110579F055
:101060000E94CB07CE01B6010E94BA070E94EF078B
:10107000CE01B7010E94AA070E94DD070AC0CE0177
:10108000B6010E94BA070E94EF07CE01B7010E9485
:10109000AA07888199810E94FD13888399838C8196
:1010A0009D810E94FD13282F392F2C833D83888139
:1010B00099818E159F0541F48A81813029F48B81B5
:1010C00090E08A159B0511F020EF3FEFC901DF91F9
:1010D000CF911F910F91FF90EF90DF90CF90BF9035
:1010E000AF900895CF92DF92EF92FF920F931F93EC
:1010F000CF93DF937C016B01EA018901A0916031FC
:10110000B09161311896ED91FC911997309739F0B3
:101110001A968D919C911B9761E070E01995C7011B
:10112000B601AE01980101E010E00E940F08E82E20
:10113000092FA0916031B09161311896ED91FC9129
:101140001997309739F01A968D919C911B9760E012
:1011500070E019958E2D902FDF91CF911F910F91F7
:10116000FF90EF90DF90CF9008954F925F926F9233
:101170007F928F929F92AF92BF92CF92DF92EF9227
:10118000FF920F931F93CF93DF935C014B013A01C2
:101190002901C0916031D0916131CE014E9669E054
:1011A00070E040E050E028E130E00E947208A114B5
:1011B000B10449F02EA13FA148A559A5F50120830E
:1011C0003183428353838114910449F02AA53BA5BE
:1011D0004CA55DA5F40120833183428353836114C0
:1011E000710449F02EA53FA548A959A9F301208310
:1011F0003183428353834114510449F02AA93BA906
:101200004CA95DA9F20120833183428353830115E8
:10121000110539F02BAD332727FD3095F8012083D8
:101220003183C114D10439F02AAD332727FD30951D
:10123000F60120833183E114F10449F02EA93FA97E
:1012400048AD59ADF7012083318342835383DF9149
:10125000CF911F910F91FF90EF90DF90CF90BF90B3
:10126000AF909F908F907F906F905F904F90089578
:10127000DF92EF92FF920F931F93FC01D02EA0916B
:101280006031B0916131009759F0E080F1800281C6
:1012900013819696ED92FD920D931C93999706C03B
:1012A00096961D921D921D921C929997611571053B
:1012B00061F0FB0160817181828193819A966D93C7
:1012C0007D938D939C939D9706C09A961D921D9237
:1012D0001D921C929D974115510561F0FA014081C4
:1012E0005181628173819E964D935D936D937C9342
:1012F000D19706C09E961D921D921D921C92D19769
:101300002115310561F0F90120813181428153813C
:10131000D2962D933D934D935C93D59706C0D2966C
:101320001D921D921D921C92D597D696DC92D6974F
:10133000CD014E9668E070E044E150E020E030E0FE
:101340000E9472081F910F91FF90EF90DF90089517
:10135000CF92DF92EF92FF920F931F93CF93DF9381
:101360006C01EB010091603110916131209709F41B
:1013700091C0CB0183709070009731F09B01237076
:10138000822F24E0281B01C020E0F80124A3CE0115
:101390000896820F911D0E94F913F801868F978F8E
:1013A00082E080A38BE181A312A213A2A0916031FD
:1013B000B09161311896ED91FC911997309739F001
:1013C0001A968D919C911B9761E070E019958EE1C2
:1013D000E82EF12CE00EF11E0E94CB07C70168E059
:1013E00070E00E94BA07F80184A1C80FD11DC601A0
:1013F000BE010E94BA078C179D07A9F00E94DD0765
:10140000A0916031B09161311896ED91FC911997DE
:10141000309709F442C01A968D919C911B9760E019
:1014200070E019953AC00E94EF07C70168E070E0CC
:101430000E94AA070E94DD07A0916031B09161313E
:101440001896ED91FC911997309739F01A968D9175
:101450009C911B9760E070E01995F801868D978D3F
:101460000E94FD13F801868F978F82A193A10E949D
:10147000FD13282F392FF80122A333A3868D978DD2
:101480008830910551F480A1833039F481A18B31EA
:1014900021F405C020E030E002C020EF3FEFC90199
:1014A000DF91CF911F910F91FF90EF90DF90CF9040
:1014B00008958F929F92AF92BF92CF92DF92EF9258
:1014C000FF920F931F93DF93CF930F92CDB7DEB7A9
:1014D0004C016B015A01790187E789838FE891E319
:1014E000809360319093613160E070E046E251E0BA
:1014F0000E942116E0916031F0916131C082D18269
:10150000A282B382E482F5820683178381E0881683
:10151000910421F480898860808B1DC00E94CB07D4
:101520008E010F5F1F4FC80161E070E00E94BA0793
:10153000C80161E070E00E94AA07E02E012F06C0FA
:101540008E2D902F61E070E00E94AA0789818E3273
:10155000B9F30E94DD0780E090E00F90CF91DF911A
:101560001F910F91FF90EF90DF90CF90BF90AF90C1
:101570009F908F9008950F931F93CF93DF938C01CB
:10158000C0916031D0916131CE014E9663E270E03E
:1015900040E050E024E030E00E9472089C0197FD9A
:1015A00005C08EA1F801808320E030E0C901DF9101
:1015B000CF911F910F910895EF92FF920F931F9378
:1015C000CF93DF93EC018B01E0916031F0916131B9
:1015D000009719F081E086A301C016A2CF014E96B4
:1015E0006FE170E044E050E020E030E00E947208DB
:1015F0007C01E0916031F0916131C087D187028731
:101600001387C80160E070E0FE011995C701DF9102
:10161000CF911F910F91FF90EF900895E09160316D
:10162000F091613184879587668777870895E09187
:101630006031F091613181E0818B08950F931F93A8
:10164000DF93CF930F92CDB7DEB700916031109149
:10165000613149830E940114F80166A377A380A732
:1016600091A7498142A780916031909161314E9656
:1016700060E070E048E050E024E030E00E94720852
:101680000F90CF91DF911F910F910895AF92BF926C
:10169000CF92DF92EF92FF920F931F93DF93CF933E
:1016A0000F920F92CDB7DEB787E78983A0916031A3
:1016B000B09161311896ED91FC911997309739F0FE
:1016C0001A968D919C911B9761E070E0199580911D
:1016D0006031909161314E9668E170E040E050E0F9
:1016E00020E030E00E9472086C0197FD2FC0E0916D
:1016F0006031F0916131808983FD28C00E94CB0761
:101700008E010F5F1F4FC80161E070E00E94BA07B1
:1017100092E0E92EF12CEC0EFD1EC70161E070E0B5
:101720000E94AA0758011E2D0F2D0BC0C50161E0B4
:1017300070E00E94BA07812F902F61E070E00E9454
:10174000AA078A81873791F70E94DD07A09160314F
:10175000B09161311896ED91FC911997309739F05D
:101760001A968D919C911B9760E070E01995C601C7
:101770000F900F90CF91DF911F910F91FF90EF90FD
:10178000DF90CF90BF90AF9008956F927F928F922D
:101790009F92AF92BF92CF92DF92EF92FF920F9300
:1017A0001F93CF93DF933C016B015A014901C09114
:1017B0006031D0916131CE014E9662E070E040E040
:1017C00050E024E230E00E9472087C0197FD3AC0AC
:1017D0008EA190E0A0E0B0E0DC01992788272FA13E
:1017E00030E040E050E0542F432F322F2227822B4D
:1017F000932BA42BB52B28A530E040E050E0822BA2
:10180000932BA42BB52BF30180839183A283B38305
:10181000C114D10451F0A114B10439F0BE01665DC8
:101820007F4FC601A5010E9430168114910451F02A
:101830000115110539F0BE01665C7F4FC401A80196
:101840000E943016C701DF91CF911F910F91FF9039
:10185000EF90DF90CF90BF90AF909F908F907F9050
:101860006F900895E0916031F0916131828B938B9C
:10187000648B758B0895AF92BF92CF92DF92EF92F7
:10188000FF920F931F93CF93DF936C017B015A015B
:101890000091603110916131E801A696CE0160E0BF
:1018A00070E048E650E00E942116C114D10431F0E6
:1018B000CE01B60141E250E00E941E16E114F1048F
:1018C00061F081E0A816B10449F1C7010E94271612
:1018D00008978833910510F113C0F801E657FF4FC0
:1018E000A08280916031909161314E9663E070E00A
:1018F00048E650E020E030E00E9472089C0102C0FF
:101900002EEF3FEFC901DF91CF911F910F91FF9013
:10191000EF90DF90CF90BF90AF900895C801865BA5
:101920009F4FB7014FE350E00E943016D6CF809111
:101930006031909161314E9664E070E040E050E09B
:1019400020E030E00E94720808950F931F9300E09A
:1019500010E00E9438091F910F910895CF92DF92F5
:10196000EF92FF920F931F9300E010E0EE24FF240C
:10197000CC24DD240E94B5081F910F91FF90EF90B9
:10198000DF90CF9008950F931F938C0180E090E03B
:1019900060E070E040E050E020E030E00E94380974
:1019A0001F910F910895CF92DF92EF92FF920F93C4
:1019B0001F938C0180E090E060E070E040E050E038
:1019C00020E030E0EE24FF24CC24DD240E94B50882
:1019D0001F910F91FF90EF90DF90CF900895E091CD
:1019E0006031F091613186A3CF014E9669E170E0DC
:1019F00044E050E020E030E00E9472080895E09159
:101A00006031F0916131868B978B608F718F089573
:101A10000F931F93CF93DF938C01C0916031D091CE
:101A20006131CE014E9666E070E040E050E024E384
:101A300030E00E9472080115110541F0BE016A5D97
:101A40007F4FC80146E050E00E941E1680E090E003
:101A5000DF91CF911F910F910895EF92FF920F9315
:101A60001F93CF93DF938C01C0916031D09161318E
:101A7000CE014E9666E070E040E050E024E330E0B6
:101A80000E9472087C010115110521F1BE01645DFF
:101A90007F4FC801819646E050E00E941E16BE01AD
:101AA0006E5C7F4FC80141E250E00E941E16FE01AD
:101AB000EA5AFF4F808191810E94FD13F80187A3AC
:101AC00090A7C85ADF4F888199810E94FD13F801C1
:101AD00081A792A7C701DF91CF911F910F91FF902E
:101AE000EF900895AF92BF92CF92DF92FF920F9343
:101AF0001F93DF93CF930F92CDB7DEB7F82E0091EF
:101B00006031109161318FE090E069830E9412167C
:101B10005C016981009779F1F801F6A267A38091D1
:101B20006031909161314E966BE070E044E050E09E
:101B300020E030E00E9472088C0197FF04C0C501CC
:101B40000E941B161AC0F5018083918313821482B0
:101B5000E0916231F0916331309731F4A0926231BB
:101B6000B09263310AC0FC01838194810097D9F758
:101B7000A382B48202C00DEF1FEFC8010F90CF9176
:101B8000DF911F910F91FF90DF90CF90BF90AF90AA
:101B900008950F931F93CF93DF93EB018A010E9467
:101BA0009907FC01009739F0C783D0870387148712
:101BB00020E030E002C02EEF3FEFC901DF91CF916E
:101BC0001F910F9108950F931F93CF93DF93EB0114
:101BD0008A010E949907FC01009739F0C187D287DA
:101BE0000587168720E030E002C02EEF3FEFC901E5
:101BF000DF91CF911F910F910895EF92FF920F9374
:101C00001F93CF93DF93EB017A0100916031109124
:101C100061310E94F913F80182A793A78881998105
:101C2000AA81BB8186A397A3A0A7B1A7C7010E94E1
:101C3000F913F80184A795A78091603190916131E3
:101C40004E966CE070E048E050E020E030E00E940A
:101C50007208DF91CF911F910F91FF90EF9008953F
:101C6000BF92CF92DF92EF92FF920F931F93CF9389
:101C7000DF93EC01B62E6A01790100916031109179
:101C800061310E949907FC010097D9F0C582D68284
:101C9000E386F4861282CE010E94F913F80186A32E
:101CA00097A3B0A680916031909161314E966DE01E
:101CB00070E044E050E020E030E00E9472089C01B7
:101CC00002C02EEF3FEFC901DF91CF911F910F911D
:101CD000FF90EF90DF90CF90BF900895CF92DF926A
:101CE000EF92FF920F931F93CF93DF93EC016B0161
:101CF0007A0100916031109161310E94990700973B
:101D000039F1FC011282CE010E94F913F80182A779
:101D100093A7F60180819181A281B381F80186A306
:101D200097A3A0A7B1A7C7010E94F913F80184A740
:101D300095A780916031909161314E966EE070E090
:101D400048E050E020E030E00E9472089C0102C0B0
:101D50002EEF3FEFC901DF91CF911F910F91FF90BF
:101D6000EF90DF90CF900895CF92DF92EF92FF92A5
:101D70000F931F93CF93DF937C01009160311091FB
:101D800061318FE090E00E941216C82EE6016E01CC
:101D9000D92EE601209771F1C7010E94F913F801CD
:101DA00086A397A380916031909161314E9664E152
:101DB00070E044E050E020E030E00E9472088C01C6
:101DC00097FF04C0C6010E941B1616C08883998322
:101DD0001B821C828A8181608A83E0916231F0914A
:101DE000633101C0FC01838194810097D9F7C383DB
:101DF000D48302C00DEF1FEFC801DF91CF911F9177
:101E00000F91FF90EF90DF90CF9008950F931F9365
:101E1000CF93DF93EC0100916031109161310E940A
:101E2000F913D80196968D939C9397978091603182
:101E3000909161314E966FE070E044E050E020E018
:101E400030E00E9472088091623190916331FC0110
:101E5000A0E0B0E02DC0208131812C173D0719F59D
:101E6000228122FD20C0C0916031D091613138893A
:101E700032FF03C0246022831DC0109751F4DC019F
:101E800013968D919C911497809362319093633156
:101E900006C08381948113968D939C931497CF01F0
:101EA0000E941B1607C0DF0133812481E32FF22F2C
:101EB000309789F680E090E0DF91CF911F910F91EC
:101EC0000895AF92BF92CF92DF92EF92FF920F935D
:101ED0001F93DF93CF9300D0CDB7DEB75B017A01BC
:101EE00000916031109161310E94F913F80186A3CD
:101EF00097A3C7010E94F913F80180A791A7A091A9
:101F00006031B09161311896ED91FC91199730973D
:101F100039F01A968D919C911B9761E070E01995AC
:101F20000E94CB0780916031909161314E9660E1C3
:101F300070E044E050E020E030E000E010E00E947B
:101F40000F088C0197FD43C0E816F906F4F1C09024
:101F50006031D09061310E94EF07C6014E9668E073
:101F600070E00E94AA077C01F601868D978D0E9481
:101F7000FD13F601868F978FF8E0EF16F10429F52F
:101F8000F60120A1243009F521A12B31F1F424A17F
:101F9000E8EFEE2EEFEFFE2EE21AF108E80EF91E42
:101FA000E016F10691F4C501B7010E94AA078C0161
:101FB0008E159F0551F4F60164A1662341F0CE0110
:101FC000019670E00E94AA0702C000EF1FEF0E9476
:101FD000DD07A0916031B09161311896ED91FC91CF
:101FE0001997309739F01A968D919C911B9760E064
:101FF00070E01995C8012396CDBFDEBFCF91DF9168
:102000001F910F91FF90EF90DF90CF90BF90AF9016
:102010000895EF92FF920F931F93CF93DF938B015D
:10202000EA01E0906031F09061310E94F913F7010C
:1020300086A397A3CE010E94F913F70180A791A769
:1020400080916031909161314E9661E170E044E0A1
:1020500050E020E030E00E947208BC0197FD0AC009
:10206000C817D9072CF0C8010E94A809BC0102C0FA
:1020700060EF7FEFCB01DF91CF911F910F91FF9028
:10208000EF900895AF92BF92CF92DF92EF92FF92BE
:102090000F931F93CF93DF935B01EA016901E090F7
:1020A0006031F09061310E94F913F70182A793A784
:1020B000CE010E94F913F70184A795A7F60180814C
:1020C0009181A281B381F70186A397A3A0A7B1A7AD
:1020D000C8010E94F913F70186A797A78091603184
:1020E000909161314E9662E170E04CE050E020E06A
:1020F00030E00E947208BC0197FD0AC0C817D907DA
:102100002CF0C5010E94A809BC0102C060EF7FEF5E
:10211000CB01DF91CF911F910F91FF90EF90DF9056
:10212000CF90BF90AF9008950F931F93CF93DF93FD
:102130008B01C0916031D09161310E94F9138EA35F
:102140009FA380916031909161314E9665E170E07E
:1021500044E050E024E030E00E947208BC0197FDAA
:1021600009C02EA13FA148A559A5F80120833183BC
:1021700042835383CB01DF91CF911F910F9108953B
:10218000CF92DF92EF92FF920F931F93CF93DF9343
:10219000EC018B016A01E0906031F09061310097B1
:1021A00059F10E9427168038910530F5E091603191
:1021B000F0916131828D938D009709F5C701869664
:1021C000BE010E94391680916031909161314E9626
:1021D0006AE070E040E850E020E030E00E947208E1
:1021E0009C0197FD0EC0E0916031F0916131028F4A
:1021F000138FC48ED58E05C02EEF3FEF02C022EFA5
:102200003FEFC901DF91CF911F910F91FF90EF90A8
:10221000DF90CF900895AF92BF92CF92DF92EF926E
:10222000FF920F931F93DF93CF93CDB7DEB72A971B
:10223000CDBFDEBF8091603190916131009709F48C
:10224000A9C14E9661E070E040E050E020E030E04F
:102250000E947208009709F49DC1809160319091AD
:1022600061314E9665E070E040E050E020E030E003
:102270000E9472080097D1F4A0916031B091613151
:102280005296ED91FC915397309761F150968C9155
:10229000509780FD27C0816050968C93509754963C
:1022A0008D919C91559761E070E01BC097FF1AC01B
:1022B000A0916031B09161315296ED91FC915397AC
:1022C000309781F050968C91509780FF0BC08E7F95
:1022D00050968C93509754968D919C91559760E0B1
:1022E00070E01995A3E0AA2EB12CAC0EBD1EC5015D
:1022F00060E070E040E050E020E030E000E010E01E
:10230000F7E0EF2EF12CEC0EFD1E6E010894C11CBF
:10231000D11C0E94B5080097D1F4A0916031B09112
:1023200061315696ED91FC915797309769F150962F
:102330008C91509781FD28C0826050968C93509765
:1023400058968D919C915997B50119951DC097FF8D
:1023500042C0A0916031B09161315696ED91FC91EF
:1023600057973097C1F150968C91509781FF33C0A9
:102370008D7F50968C93509758968D919C9159973C
:1023800060E070E0199527C0A0916031B091613193
:102390005A96ED91FC915B973097E9F089819A818B
:1023A000009741F45C968D919C915D97BE01695FA9
:1023B0007F4F0AC02FEF8F3F920769F45C968D9193
:1023C0009C915D9760E070E01995E0916031F0912B
:1023D0006131128E138EE0916031F091613180890C
:1023E0008460808B009162311091633193C0D80179
:1023F0008D919C910E94F913F70186A397A3809178
:102400006031909161314E9663E170E044E050E0BC
:1024100024E030E00E947208AC0197FD22C0D70191
:1024200096968C9196978130D1F4F801928190FD27
:1024300042C00780F085E02D3097E9F1892F816057
:102440008D7FD80112968C9312976D917C91119784
:102450001B968D919C911C9741E050E057C08430B1
:10246000B9F4F801828181FD25C00780F085E02D57
:10247000309701F18E7F8260D80112968C9312976B
:102480006D917C9111971B968D919C911C973CC0EE
:10249000833089F4D8011596ED91FC911697309709
:1024A00051F06D917C9111971B968D919C911C9789
:1024B00019952DC084E0141615067CF4D8011996E0
:1024C000ED91FC911A97309741F06D917C911197A5
:1024D0001D968D919C911E9719C08823C1F4F80117
:1024E000828180FF14C00184F285E02D309779F05D
:1024F0008E7FD80112968C9312976D917C911197D3
:102500001D968D919C911E9740E050E01995F80121
:1025100003811481E0906031F09061310115110563
:1025200009F065CFD70150968C9150978B7F5096CC
:102530008C935097E0916231F091633100E010E0AC
:1025400027C0828182FF1FC00115110569F4A09187
:102550006231B091633113968D919C911497809361
:1025600062319093633107C083819481D8011396BF
:102570008D939C931497A380E480CF010E941B1637
:102580009A2D8E2D03C08F0193818481E92FF82F1E
:102590003097B9F62A96CDBFDEBFCF91DF911F915C
:1025A0000F91FF90EF90DF90CF90BF90AF90089584
:1025B000E0916031F091613186A3CF014E9666E1E2
:1025C00070E044E050E020E030E00E94720808959E
:1025D0000F931F93CF93DF938C01C0916031D09103
:1025E0006131CE014E966AE170E040E050E024E0B7
:1025F00030E00E9472089C0197FD03C08EA1F80193
:102600008083C901DF91CF911F910F910895E091CF
:102610006031F091613186A3CF014E9667E170E0A1
:1026200044E050E020E030E00E9472080895E0911C
:102630006031F091613121E0009709F420E026A398
:10264000CF014E966EE170E044E050E020E030E0D3
:102650000E94720808958F929F92AF92BF92CF927C
:10266000DF92EF92FF920F931F93CF93DF93F82E99
:102670004A015B01C901B801C0916031D09161315B
:102680000E9401146EA37FA388A799A7C501B40176
:102690000E9401146AA77BA78CA79DA7C6010E9470
:1026A000F9138EA79FA7F8AAE9AA809160319091AB
:1026B00061314E966DE170E04FE050E020E030E097
:1026C0000E947208DF91CF911F910F91FF90EF90C0
:1026D000DF90CF90BF90AF909F908F900895FF9222
:1026E0000F931F93CF93DF93F82EC901C0916031F0
:1026F000D09161314EA35FA368A779A70E94F91317
:102700008AA79BA7FCA60115110579F0C8010E94B4
:1027100027168F379105C0F4C8010E942716AC0117
:10272000CE018E96B8010E941E1680916031909164
:1027300061314E966CE170E048E850E020E030E016
:102740000E9472089C0102C02EEF3FEFC901DF9189
:10275000CF911F910F91FF900895E0916031F0911A
:10276000613121E0009709F420E026A3CF014E96C5
:1027700060E270E044E050E020E030E00E94720847
:102780000895CF93DF93C0916031D09161310E9461
:1027900001146EA37FA388A799A7809160319091BF
:1027A00061314E9661E270E044E050E020E030E0BC
:1027B0000E947208DF91CF910895CF93DF93C0916B
:1027C0006031D09161310E9401146EA37FA388A76C
:1027D00099A780916031909161314E9662E270E0EC
:1027E00044E050E020E030E00E947208DF91CF9199
:1027F0000895382F292FC9010895382F292FC9018D
:102800000895AF92BF92CF92DF92EF92FF920F9313
:102810001F93292F332744275527162F0027FF24DE
:10282000EE242E293F29402B512BEE24F62E072F84
:10283000182FA12CB12CFFEFCF2ED12CEA20FB209A
:102840000C211D212E293F29402B512B672F782F3A
:10285000892F9927607080709070262B372B482B1A
:10286000592BB901CA011F910F91FF90EF90DF9092
:10287000CF90BF90AF9008950E94011408952F92B9
:102880003F924F925F926F927F928F929F92AF9200
:10289000BF92CF92DF92EF92FF920F931F93DF933D
:1028A000CF93CDB7DEB76097CDBFDEBFDC011B0194
:1028B0000C91112707FD10958DE0482E512C4C0EE0
:1028C0005D1E5E010894A11CB11C802F80538A30CC
:1028D00008F028C100331105A1F411960C911127BD
:1028E00007FD10950837110519F00835110569F431
:1028F00011960C91112707FD1095F0E1CF2ED12CE8
:1029000007C0EAE0CE2ED12C03C078E0C72ED12C30
:102910007D010894E11CF11C60E070E0CB01360100
:10292000882477FC8094982CF7013197202F302F42
:1029300030533A30A0F4A40193010E941E509B0131
:10294000AC0100531040B801882777FD8095982F7F
:10295000620F731F841F951FD7010C912BC0B0E12C
:10296000CB16D10471F5A02FA156A63020F0302F40
:102970003154363030F59B01AC0164E0220F331F37
:10298000441F551F6A95D1F7065F1F4FAA3118F4EF
:1029900081E690E002C081E490E0081B190BB801C9
:1029A000882777FD8095982F622B732B842B952B8E
:1029B000F7010081112707FD10950894E11CF11C17
:1029C000B3CF0E32110589F4A414B50409F4AAC0DA
:1029D000D5016D937D938D939D935D01DF011196DC
:1029E0000181112707FD109570CF01151105C1F068
:1029F000203208F497C007FD95C00032110581F020
:102A00000C30110569F00A30110551F00D30110537
:102A100039F00930110521F00B30110509F082C0A1
:102A20009E012F5F3F4FA21AB30AB594A794B594A5
:102A3000A7940894A11CB11CB2E0AB16B10499F0A4
:102A4000E3E0AE16B1042CF4A114B10409F46AC099
:102A50005EC0F3E0AF16B104C1F024E0A216B104E9
:102A600009F055C02BC0603030E0730730E08307B9
:102A700031E0930708F056C029813A814B815C818F
:102A8000522F4427332722273EC06030A0E07A0728
:102A9000A1E08A07A0E09A0708F044C02D813E819A
:102AA0004F815885A90133272227E980FA800B81BD
:102AB0001C811E2D0027FF24EE2421C06F3F7105CD
:102AC0008105910509F070F52D813E814F81588572
:102AD000A90133272227E980FA800B811C811E2D52
:102AE0000027FF24EE242E293F29402B512BE98477
:102AF000FA840B851C85102F0F2DFE2CEE242E2919
:102B00003F29402B512B622B732B842B952B2114A7
:102B1000310459F00E940114F101608371838283B2
:102B2000938303C020E030E002C021E030E0C9011F
:102B30006096CDBFDEBFCF91DF911F910F91FF90C7
:102B4000EF90DF90CF90BF90AF909F908F907F904D
:102B50006F905F904F903F902F900895AF92BF92EB
:102B6000DF92EF92FF920F931F93DF93CF93CDB736
:102B7000DEB72797CDBFDEBFFC0180819181A281A6
:102B8000B3818C839D83AE83BF83DE011496AD0138
:102B90004C5F5F4F34E6A32E31E3B32E2AE0D22EF2
:102BA0009E012F5F3F4F9EE2E92E8C91FF246D2DF9
:102BB0000E943D5089010F0D111D905DF801908319
:102BC000F3948823A1F76F2D1D92C50109C0FA94D3
:102BD00089010F0D111DF8017081FC017193CF0166
:102BE000FF20A9F7C501860F911DFC01E1925F014D
:102BF000A417B507D1F6FC01108284E691E327966D
:102C0000CDBFDEBFCF91DF911F910F91FF90EF906D
:102C1000DF90BF90AF90089580E090E008950E940B
:102C2000D2500895BC0181E090E00E94AD5008951B
:102C30000E94055208950E946C5108950E94775495
:102C400008950E94925408950E9480540895FC01B2
:102C500001900020E9F73197E81BF90BCF010895A7
:102C60000E94D55408950E94C75408950E94B754F5
:102C700008950E94C05408950E9443540895CF922D
:102C8000DF92EF92FF920F931F93CF93DF937C011C
:102C90008B01CB0101960E94D250C82EE6016E0135
:102CA000D92EE601209749F0C601B701A8010E947C
:102CB000D554F601E00FF11F1082CE01DF91CF91C4
:102CC0001F910F91FF90EF90DF90CF9008950E9499
:102CD0006A5408950E94DE5208950E94AC540895EB
:102CE0000E94E45408950E94995408950E94EF545C
:102CF0000895DF93CF93CDB7DEB7FE013C968E816A
:102D00009F81688579854A855B859F010E9466550C
:102D1000CF91DF9108950E9466550895AF92BF92BA
:102D2000CF92DF92EF92FF920F931F93DF93CF9397
:102D3000CDB7DEB78E01025F1F4FF801A190B190B1
:102D40008F0180EA90E00E94D250D82EC92EE82E42
:102D5000F92EE114F104E9F0C70160EA70E0A50181
:102D600098010E9466558C0197FD04C0C601C92ECA
:102D7000D82E06C0C7010E946C510BC00E940246AB
:102D8000F60181916F018823C9F7C7010E946C5138
:102D900002C00FEF1FEFC801CF91DF911F910F917C
:102DA000FF90EF90DF90CF90BF90AF900895CF93BA
:102DB000DF939C01009741F420917431309175317B
:102DC0002115310509F440C0F9019F01819199272E
:102DD00087FD90957E2F6F2FA0E0B0E203C084178F
:102DE000950799F34D91552747FD5095411551058C
:102DF000B1F7009739F4109274311092753120E0D8
:102E000030E022C0CB01E92FF62FEF014191552789
:102E100047FD5095CF01A0E0B0E26D91772767FDA7
:102E200070956417750761F44115510511F018820A
:102E300002C080E090E0809374319093753104C0BB
:102E40006115710551F7E1CFC901DF91CF91089567
:102E5000CF93DF93EC01009749F08A859B8500971B
:102E600011F00E941B16CE010E941B16DF91CF911C
:102E70000895CF93DF93FC01DB0116964D935C938D
:102E80001797C281D381209721F46283738307C08F
:102E9000EC01888599850097D9F7A887B987189696
:102EA0001D921C921997DF91CF910895FB014683E3
:102EB0005783FC0166A777A70895FC018081918163
:102EC0000895CF92DF92EF92FF920F931F93CF93CB
:102ED000DF937C016A01062F172FC0E0D0E011C0FC
:102EE000D8016D918D01772767FD7095D7011696F2
:102EF000ED91FC91179718968D919C9119971995C2
:102F00002196CC15DD0564F3DF91CF911F910F91D0
:102F1000FF90EF90DF90CF900895AF92BF92CF9245
:102F2000DF92EF92FF920F931F93DF93CF93CDB772
:102F3000DEB7AE84BF848E010E5E1F4F80E590E049
:102F40000E940F166C017C01009721F160E570E092
:102F50004889598998010E948B168C0197FF11C0EE
:102F6000C6010E941B1616C0772767FD7095D50114
:102F70001696ED91FC91179718968D919C91199743
:102F80001995F60161916F01662371F7C7010E94DF
:102F90001B1602C00DEF1FEFC801CF91DF911F91EB
:102FA0000F91FF90EF90DF90CF90BF90AF9008957A
:102FB000EF92FF920F931F93CF93DF938C01DC016D
:102FC0001296CD91DC91139783E0E82E80E2F82EE3
:102FD00024C0288139818C819D81009711F482E081
:102FE00090E2EDB7FEB73897EDBFFEBF3196ADB7B3
:102FF000BEB711960D931C931297E282F38224833D
:103000003583868397830E948D170884D985C02DC8
:10301000EDB7FEB73896EDBFFEBF2097D1F6DF9132
:10302000CF911F910F91FF90EF9008952F923F92B3
:103030004F925F926F927F928F929F92AF92BF92C8
:10304000CF92DF92EF92FF920F931F93DF93CF9374
:10305000CDB7DEB7C655D040CDBFDEBF65968EAFCB
:103060009FAF65971A0149012DB73EB728503040F0
:103070002DBF3EBFEDB7FEB73196ADB7BEB71196C7
:103080008D939C9312978EE090E282839383648366
:103090007583868297820E948D17EDB7FEB73896AA
:1030A000EDBFFEBFEE24FF249E012F5A3F4F6796CF
:1030B0002EAF3FAF67972E010894411C511C87012A
:1030C000B1C08DB79EB708978DBF9EBFEDB7FEB755
:1030D0003196ADB7BEB711964D925C92129720E52E
:1030E00030E02283338386E290E2848395830683F3
:1030F00017830E947916D201A80FB91F6396AEAF4D
:10310000BFAF63973801EDB7FEB73896EDBFFEBF8E
:103110006801AA24BB2478018D01C814D9044CF598
:103120002DB73EB7285030402DBF3EBFEDB7FEB79C
:103130003196ADB7BEB711960D931C931297679653
:103140008EAD9FAD6797801B910B828393832DE299
:1031500030E224833583D101AC0DBD1D8C91868373
:1031600017820E9479168DB79EB708968DBF9EBFB5
:1031700005C0C80163E370E20E9439160D5F1F4F5E
:103180000894A11CB11C0894C11CD11C90E1A91683
:10319000B10419F687016396EEACFFAC6397A0E328
:1031A000B0E0EA0EFB1EC70167E370E20E94391629
:1031B00080E090E0F7016814790474F4D101A60D61
:1031C000B71D4C919F012F5F3F4F403214F0408359
:1031D00002C0BEE2B083F90101960894611C711C23
:1031E0008031910541F7108200D000D0EDB7FEB7D5
:1031F000319665962EAD3FAD6597ADB7BEB71196CA
:103200002D933C9312978AE390E2828393834482C6
:1032100055820E948D17005F1F4FADB7BEB716963F
:10322000ADBFBEBF081519050CF44BCFCA5ADF4F0E
:10323000CDBFDEBFCF91DF911F910F91FF90EF9037
:10324000DF90CF90BF90AF909F908F907F906F90C6
:103250005F904F903F902F9008956F927F928F9242
:103260009F92AF92BF92CF92DF92EF92FF920F9315
:103270001F93DF93CF930F92CDB7DEB73C01DC01F4
:1032800050968D919C9151970097B9F11E968D9112
:103290009C911F978F3491052CF050961D921C9293
:1032A0005197AEC16E3671F0623719F06C35E1F4AA
:1032B00013C0D3011A96ED91FC911B97E80FF91FEB
:1032C0008DE008C0D3011A96ED91FC911B97E80F91
:1032D000F91F8AE0808308C0D3011A96ED91FC9112
:1032E0001B97E80FF91F6083F30186859785019688
:1032F00086879787108A118A83C16A30E1F16B3023
:1033000024F4683009F038C112C06D30A1F16C3579
:1033100009F032C1D30152968C91529782FF07C0B7
:1033200081E090E050968D939C93519769C1F30191
:1033300086859785009709F463C1828981FD14C051
:1033400000D00F92ADB7BEB711966D927C921297D6
:1033500082E490E213968D939C9314970E948D17AC
:103360000F900F900F900F90F3018685978501972E
:103370008687978745C1D3011A96ED91FC911B97DB
:103380001E968D919C911F97E80FF91F10825296FF
:103390008C91529781FD10C000D00F92EDB7FEB70F
:1033A0006182728286E490E2838394830E948D1707
:1033B0000F900F900F900F90D3011A968D919C91C2
:1033C0001B9754961D921C92559722E030E2569618
:1033D0002D933C93579717C0F30124893589F90140
:1033E0003B96EE0FFF1FE60DF71D80839183C90109
:1033F0000196D30154968D939C9355978C309105EB
:1034000031F080E090E00E94D716009729F7F30191
:10341000C688D788C6010E942716009709F447C0BE
:10342000D30112960D911C911397AA24BB24EE246C
:10343000FF2421C0F80180819181B6010E943616D7
:10344000009719F1D8018D909C90C6010E94271613
:10345000AC01C401B6010E943316009749F4E1148F
:10346000F10411F4780104C0780191E0A92EB12C87
:10347000F8010085118501151105E1F6A114B104CB
:10348000B1F4E114F10499F08701D80116968D91F9
:103490009C911797F3018083918364897589A301B7
:1034A0004A5E5F4F1296ED91FC91139716C0D301BF
:1034B0009E96ED91FC919F97309791F08681978130
:1034C0008D939C93119754966D917C915597A30180
:1034D0004A5E5F4F0280F381E02DC301199524C03D
:1034E000F301868997890E9427160097E9F000D09A
:1034F00000D0EDB7FEB73196ADB7BEB711966D925D
:103500007C92129789E490E282839383D30156964A
:103510008D919C915797848395830E948D17EDB769
:10352000FEB73696EDBFFEBFD3011E961D921C92CC
:103530001F9752968C91529780FD62C000D000D0A8
:10354000EDB7FEB73196ADB7BEB711966D927C92CE
:10355000129780E690E282839383D30114968D9133
:103560009C911597848395830E948D17EDB7FEB7C4
:103570003696EDBFFEBF44C0D3011E968D919C913F
:103580001F978F349105E4F5862F80528F35C0F553
:1035900052968C91529781FD1EC000D000D0EDB79D
:1035A000FEB73196ADB7BEB711966D927C92129769
:1035B00084E690E282839383862F992787FD9095F6
:1035C0008483958369830E948D17EDB7FEB7369685
:1035D000EDBFFEBF6981D3011A96ED91FC911B9757
:1035E0001E968D919C911F97E80FF91F60831E9680
:1035F0008D919C911F9701961E968D939C931F977A
:103600000F90CF91DF911F910F91FF90EF90DF907E
:10361000CF90BF90AF909F908F907F906F900895C4
:103620006F927F928F929F92AF92BF92CF92DF92D2
:10363000EF92FF920F931F93CF93DF937C016B0167
:103640004A01B22EA32E6115710509F455C080E31D
:1036500090E00E940F16682EE3013E01792EE301EF
:103660008301209709F44AC0C30160E070E040E3A1
:1036700050E00E942116E114F10421F457E6E52EF2
:1036800050E2F52EEC82FD8280E590E08C879D87EC
:103690000E940F168A879B87009721F4CE010E9413
:1036A0001B162AC04C855D8560E070E00E942116E3
:1036B000BA8AAB8ACE82DF8288869986B0FC1EC029
:1036C00000D000D0EDB7FEB73196ADB7BEB71196BA
:1036D000CD93DC93129780E690E2828393838C8172
:1036E0009D81848395830E948D172DB73EB72A5FF5
:1036F0003F4F2DBF3EBF02C000E010E0C801DF9188
:10370000CF911F910F91FF90EF90DF90CF90BF90DE
:10371000AF909F908F907F906F9008952F923F92DF
:103720004F925F926F927F928F929F92AF92BF92D1
:10373000CF92DF92EF92FF920F931F93DF93CF937D
:103740000F920F92CDB7DEB75C0181E090E0698304
:103750007A830E941216282E392E69817A812114CB
:10376000310409F44CC0062F172FEE24FF24250145
:103770000894410851083FC061E0C62ED12CE414E2
:10378000F50414F0CC24DD24C1010E9427164C015D
:103790003801F801808191810E942716B6016F5F80
:1037A0007F4F680D791D680F791FC1010E9418169F
:1037B000009731F4C1010E941B16222433241FC03C
:1037C0001C010E9427160E5F1F4FF301608171815B
:1037D000820D931D0E943916C114D10449F0C10114
:1037E0000E942716820D931D60E070E20E94391638
:1037F0000894E11CF11CEA14FB040CF4BDCFC101D8
:103800000F900F90CF91DF911F910F91FF90EF904C
:10381000DF90CF90BF90AF909F908F907F906F90F0
:103820005F904F903F902F9008952F923F924F922C
:103830005F926F927F928F929F92AF92BF92CF9240
:10384000DF92EF92FF920F931F93DF93CF93CDB749
:10385000DEB7C455D040CDBFDEBF1B014A0100D04A
:1038600000D0EDB7FEB7319625E830E2ADB7BEB770
:1038700011962D933C9312978283938344835583AF
:103880000E948E16EDB7FEB73696EDBFFEBFEE2452
:10389000FF249E012F5A3F4F65962EAF3FAF65978D
:1038A0002E010894411C511C8701A5C08DB79EB7FD
:1038B00008978DBF9EBFEDB7FEB73196ADB7BEB7C7
:1038C00011964D925C92129720E530E0228333836B
:1038D0008DE990E284839583068317830E9479168D
:1038E000D201A80FB91F6396AEAFBFAF639738017F
:1038F000EDB7FEB73896EDBFFEBF6801AA24BB2422
:1039000078018D01C814D9044CF52DB73EB7285065
:1039100030402DBF3EBFEDB7FEB73196ADB7BEB755
:1039200011960D931C93129765968EAD9FAD65977A
:10393000801B910B8283938324EA30E224833583B6
:10394000D101AC0DBD1D8C91868317820E94791622
:103950008DB79EB708968DBF9EBF05C0C8016AEAA5
:1039600070E20E9439160D5F1F4F0894A11CB11C14
:103970000894C11CD11C90E1A916B10419F6870165
:103980006396EEACFFAC6397A0E3B0E0EA0EFB1EDB
:10399000C7016EEA70E20E94391680E090E0F701FC
:1039A0006814790474F4D101A60DB71D4C919F01E0
:1039B0002F5F3F4F403214F0408302C0BEE2B0831D
:1039C000F90101960894611C711C8031910541F741
:1039D000108200D00F9221EB30E2EDB7FEB72183C9
:1039E0003283438254820E948E16005F1F4F0F90D5
:1039F0000F900F900F90081519050CF457CFCC5A63
:103A0000DF4FCDBFDEBFCF91DF911F910F91FF90B0
:103A1000EF90DF90CF90BF90AF909F908F907F906E
:103A20006F905F904F903F902F900895FC0197FF0B
:103A30000BC07696E631F10550F4EE0FFF1FEF5004
:103A4000FF4C2081318105C029EB30E202C021EC1E
:103A500030E2C901089586E090E00E94121680933A
:103A6000763190937731009719F42DEF3FEF02C034
:103A700020E030E0C9010895CF92DF92EF92FF92EB
:103A80000F931F93CF93DF936C018B01EA017901B0
:103A90002097A1F18CE090E00E941216FC019C019D
:103AA000009771F1C283D383E482F5820115110579
:103AB00029F086819781826086839783C0917631D1
:103AC000D0917731A881B981109721F4E883F983E7
:103AD00009C0DC018D919C9111970097D1F7ED936E
:103AE000FC9311978A819B8180879187C286D386B8
:103AF000868197818E7F8683978302C020E030E0A5
:103B0000C901DF91CF911F910F91FF90EF90DF904E
:103B1000CF900895CF93DF930097D1F1A0917631A4
:103B2000B091773114962C91149720FF0BC0DC01D3
:103B300016962D913C911797246016962D933C93E1
:103B4000179726C0CD91DC9111979E01E0E0F0E03F
:103B500019C02817390731F0F90150814181252F0B
:103B6000342F10C0309731F4288139812D933C9344
:103B7000119705C0DC012D913C91208331830E9477
:103B80001B1606C02115310521F72EEF3FEF02C0AD
:103B900020E030E0C901DF91CF910895FC01A091B0
:103BA0007631B091773112968D919C9113978087E1
:103BB000918762877387868197818E7F86839783BB
:103BC0000895E0917631F091773122813381C901F6
:103BD0000895E0917631F0917731309731F022817C
:103BE0003381280F391F22833383089541155105EE
:103BF00019F086179707A1F06817790740F0681B3E
:103C0000790B21E030E06417750760F409C08095F6
:103C10009095860F971F21E030E08417950710F4E8
:103C200020E030E0C90108950F931F93CF93DF93F5
:103C3000E0917631F0917731848195818160848340
:103C40009583C081D18130C00E811F81C8018570EC
:103C50009070009731F5E0917631F0917731628183
:103C600073814A855B85888599850E94F61D00973A
:103C7000C1F001600E831F836C817D81EA81FB812D
:103C8000CE0119958E819F8181FF0BC0E091763125
:103C9000F091773122813381288739878E7F8E8317
:103CA0009F830990D881C02D209771F6E0917631DD
:103CB000F0917731848195818E7F84839583019003
:103CC000F081E02DC0E0D0E024C0868182FF1CC0DE
:103CD000209779F42091763130917731D9018D9107
:103CE0009C91DC018D919C91D9018D939C931197AE
:103CF00004C0808191818883998310810181CF01E3
:103D00000E941B16C80103C0EF0190818181E92F39
:103D1000F82F3097D1F6DF91CF911F910F91089531
:103D2000EF92FF920F931F93CF93DF938C01C0917B
:103D30007631D0917731EA80FB806A817B81C7013F
:103D4000A8010E94F61D0097C1F3DF91CF911F914A
:103D50000F91FF90EF9008956817790730F49C0158
:103D600020953095260F371F03C09B01281B390B68
:103D7000C9010895CF93DF93FC01DB018D939C93E0
:103D8000DC0120E030E026C0863271F41082241776
:103D90003507FCF4E901CC0FDD1FCC0FDD1FC60F8A
:103DA000D71FA883B98315C08D3399F4E901CC0FCF
:103DB000DD1FCC0FDD1FC60FD71F888199810097AB
:103DC00041F010822417350724F4AA83BB832F5FA8
:103DD0003F4F31968D918823B9F6C901DF91CF917C
:103DE0000895AF92BF92CF92DF92EF92FF920F931E
:103DF0001F93CF93DF935C016A01E62EE7017E01FA
:103E0000F72EE701EE24FF2400E010E00FC06881E8
:103E100079816115710569F0C5010E943616009718
:103E200011F4EA80FB800F5F1F4F24960C151D05CF
:103E300074F3C701DF91CF911F910F91FF90EF9025
:103E4000DF90CF90BF90AF9008958DE290E061E059
:103E500070E00E9435468EE290E062E070E00E94E1
:103E600035468EE290E00E94744689E290E062E07E
:103E700070E00E94354689E290E00E945F4684EF40
:103E800091E00E94F44589E290E00E94744684EF3C
:103E900091E00E94F44580E090E0089589E290E08E
:103EA00062E070E00E94354689E290E00E945F4641
:103EB00080E090E008952DB73EB72A5030402DBFE6
:103EC0003EBFEDB7FEB73196ADB7BEB711968D9335
:103ED0009C93129787EF91E28283938381E090E035
:103EE0008483958383E090E0868397831086118690
:103EF0000E948D172DB73EB7265F3F4F2DBF3EBFA7
:103F000008952DB73EB7285030402DBF3EBFEDB7C6
:103F1000FEB73196ADB7BEB711968D939C931297AD
:103F20008DE092E282839383648375834683578313
:103F30000E948D172DB73EB7285F3F4F2DBF3EBF64
:103F40000895EF92FF920F931F93DF93CF930F92F9
:103F50000F92CDB7DEB78C017B01BE016F5F7F4F43
:103F600040E050E00E946A16F7016083718382830B
:103F7000938321E030E040E050E089819A8180170E
:103F8000910719F420E030E0A901B901CA010F90AE
:103F90000F90CF91DF911F910F91FF90EF900895B7
:103FA000CF92DF92EF92FF920F931F93DF93CF9305
:103FB00000D00F92CDB7DEB76C01623071050CF402
:103FC00042C0DA0112968D919C911397BE016F5FEA
:103FD0007F4F0E94A11F611571058105910599F11F
:103FE00069817A818B819C810E94DD138C0197FD10
:103FF00005C09EE2E92E92E2F92E04C081E3E82E8C
:1040000082E2F82EC8010E94161DEDB7FEB73A975E
:10401000EDBFFEBF3196ADB7BEB71196CD92DC9223
:10402000129725E332E222833383E482F58206830A
:104030001783808791870E948D17EDB7FEB73A9658
:10404000EDBFFEBF14C000D00F92ADB7BEB7119642
:10405000CD92DC92129782E492E213968D939C9318
:1040600014970E948D170F900F900F900F90249629
:10407000CDBFDEBFCF91DF911F910F91FF90EF90E9
:10408000DF90CF900895EF92FF920F931F93DF93ED
:10409000CF930F920F92CDB7DEB78C017B01BE019B
:1040A0006F5F7F4F40E050E00E946A16F701608327
:1040B000718321E030E089819A818017910711F4A2
:1040C00020E030E0C9010F900F90CF91DF911F9158
:1040D0000F91FF90EF900895EF92FF920F931F932F
:1040E000DF93CF930F920F92CDB7DEB78C017B0198
:1040F000BE016F5F7F4F40E050E00E946A16298149
:104100003A812017310741F077FD06C0F70160833F
:10411000718321E030E002C020E030E0C9010F905F
:104120000F90CF91DF911F910F91FF90EF90089525
:10413000CF92DF92EF92FF920F931F93DF93CF9373
:1041400000D00F92CDB7DEB76C01623071050CF470
:1041500060C0DA0112968D919C911397BE016F5F3A
:104160007F4F0E94A11F611571058105910509F41A
:1041700050C069817A818B819C810E94C1138C011E
:1041800000D000D0EDB7FEB73196ADB7BEB71196EF
:10419000CD92DC9212978AE692E2828393838981A0
:1041A0009A81848395830E948D17EDB7FEB736966A
:1041B000EDBFFEBF17FD05C03EE2E32E32E2F32E57
:1041C00004C021E3E22E22E2F22EC8010E94161D55
:1041D0002DB73EB72A5030402DBF3EBFEDB7FEB7DA
:1041E0003196ADB7BEB71196CD92DC92129725E30A
:1041F00032E222833383E482F58206831783808749
:1042000091870E948D17EDB7FEB73A96EDBFFEBFBE
:1042100014C000D00F92ADB7BEB71196CD92DC920C
:10422000129786E792E213968D939C9314970E94BF
:104230008D170F900F900F900F902496CDBFDEBF7B
:10424000CF91DF911F910F91FF90EF90DF90CF9072
:104250000895CF92DF92EF92FF920F931F93DF9317
:10426000CF930F920F92CDB7DEB76C01623071051C
:10427000ECF1DA0112968D919C911397BE016F5F5C
:104280007F4F0E944320009789F189819A810E9483
:10429000AD138C0197FD05C05EE2E52E52E2F52ECE
:1042A00004C041E3E42E42E2F42EC8010E94161D30
:1042B000EDB7FEB73A97EDBFFEBF3196ADB7BEB7CB
:1042C0001196CD92DC92129725E332E2228333835A
:1042D000E482F58206831783808791870E948D1779
:1042E000EDB7FEB73A96EDBFFEBF14C000D00F92F7
:1042F000ADB7BEB71196CD92DC92129783E992E2E8
:1043000013968D939C9314970E948D170F900F9086
:104310000F900F900F900F90CF91DF911F910F9101
:10432000FF90EF90DF90CF9008958F929F92AF9281
:10433000BF92CF92DF92EF92FF920F931F93DF9382
:10434000CF9300D00F92CDB7DEB74C017B018A012D
:104350006E010894C11CD11CC60160E070E040E011
:1043600050E020E030E00E94AE0CC701019785309C
:10437000910508F09EC021E0E216F10409F4AEC0F8
:10438000D80112968D919C9113976BEA72E20E946C
:104390003616009709F08DC0B2E0EB16F10409F46F
:1043A0009DC0F80184819581B6010E943F14009759
:1043B00009F47FC0F3E0EF16F10409F48FC0D801CF
:1043C00016968D919C91179760E070E04AE050E05E
:1043D0000E946A165B01B5E0EB16F10421F4F801C6
:1043E000E084F18402C0EE24FF2449815A816B816C
:1043F0007C8180E0950187010E946F138C0197FDFD
:1044000005C0FEE2CF2EF2E2DF2E04C0E1E3CE2EA5
:10441000E2E2DE2EC8010E94161D2DB73EB72A50DB
:1044200030402DBF3EBFEDB7FEB73196ADB7BEB73A
:1044300011968D929C92129725E332E22283338368
:10444000C482D58206831783808791870E948D1747
:10445000EDB7FEB73A96EDBFFEBFCE0101960E94C2
:10446000AE15E114F10421F47AEAE72E72E2F72E98
:104470002DB73EB72A5030402DBF3EBFEDB7FEB737
:104480003196ADB7BEB711968D929C92129725EBDF
:1044900032E22283338384839583A682B782E086C7
:1044A000F1860E948D17EDB7FEB73A96EDBFFEBFBD
:1044B0001AC000D00F92ADB7BEB711968D929C92E4
:1044C00012978DEC92E213968D939C9314970E9411
:1044D0008D170F900F900F900F9005C060E9A62EDA
:1044E0006FE1B62E80CF2496CDBFDEBFCF91DF9196
:1044F0001F910F91FF90EF90DF90CF90BF90AF9002
:104500009F908F9008950F931F938C0161157105F3
:10451000A9F400D00F92EDB7FEB73196ADB7BEB794
:1045200011968C93118381E193E2828393830E949D
:104530008D170F900F900F900F901AC0CB010E9413
:10454000AE1500D000D0EDB7FEB73196ADB7BEB70F
:1045500011960C9311832DE233E2228333838483FB
:1045600095830E948D178DB79EB706968DBF9EBF0F
:104570001F910F9108950F931F93DF93CF93CDB7A2
:10458000DEB76097CDBFDEBF8C01CE010196BE01C4
:104590006B5F7F4FAE01475F5F4F9E01235F3F4FD1
:1045A0000E94AE0C97FD03C02EE232E202C021E36E
:1045B00032E24DB75EB7485050404DBF5EBFEDB7D9
:1045C000FEB73196ADB7BEB711960D931C931297F7
:1045D0004FE353E242835383248335838683978357
:1045E0000E948D174DB75EB7485F5F4F4DBF5EBFEE
:1045F000CE0101960E94AE1500D000D0EDB7FEB7F7
:104600003196ADB7BEB711960D931C93129727E460
:1046100033E222833383848395830E948D174DB7C1
:104620005EB74A5F5F4F4DBF5EBFCE0105960E94E9
:10463000AE1500D000D0EDB7FEB73196ADB7BEB71E
:1046400011960D931C9312972EE433E22283338349
:10465000848395830E948D174DB75EB74A5F5F4F85
:104660004DBF5EBFCE0109960E94AE1500D000D0AE
:10467000EDB7FEB73196ADB7BEB711960D931C934B
:10468000129727E533E222833383848395830E9444
:104690008D174DB75EB74A5F5F4F4DBF5EBFCE010E
:1046A0000D960E94AE1500D000D0EDB7FEB7319642
:1046B000ADB7BEB711960D931C9312972EE533E25A
:1046C00022833383848395830E948D174DB75EB711
:1046D0004A5F5F4F4DBF5EBF6096CDBFDEBFCF91DB
:1046E000DF911F910F910895CF92DF92EF92FF9289
:1046F0000F931F93DF93CF930F92CDB7DEB76C016B
:10470000CE0101960E94BB0A8C0197FD05C0BEE256
:10471000EB2EB2E2FB2E04C0A1E3EA2EA2E2FA2EB7
:10472000C8010E94161D2DB73EB72A5030402DBF3C
:104730003EBFEDB7FEB73196ADB7BEB71196CD927D
:10474000DC92129725E332E222833383E482F582FE
:1047500006831783808791870E948D170F900F9093
:104760000F900F90EDB7FEB73196ADB7BEB711966B
:10477000CD92DC92129788E693E2828393838981BB
:10478000848315820E948D172DB73EB72A5F3F4F55
:104790002DBF3EBF0F90CF91DF911F910F91FF90E2
:1047A000EF90DF90CF900895CF92DF92EF92FF923B
:1047B0000F931F93DF93CF93CDB7DEB7A497CDBFF1
:1047C000DEBF6C01CE010196BE016B5F7F4F40E101
:1047D00050E09E012B5E3F4F00E110E00E94C50BB0
:1047E0008C0197FD05C09EE2E92E92E2F92E04C0ED
:1047F00081E3E82E82E2F82EC8010E94161D2DB733
:104800003EB72A5030402DBF3EBFEDB7FEB73196C0
:10481000ADB7BEB71196CD92DC92129725E332E286
:1048200022833383E482F58206831783808791870E
:104830000E948D1789819A81AB81BC810F920F9262
:104840006DB77EB76F5F7F4FEDB7FEB7C182D28283
:104850002EE733E2FB01228333832A2F30E02483C7
:104860003583292F3A2F4B2F5527307026833783D6
:10487000907080879187CE010596828793870E94EA
:104880008D172DB73EB7245F3F4F2DBF3EBF8E0122
:104890000B5E1F4FC8010E942716009711F406E710
:1048A00013E200D000D0EDB7FEB73196ADB7BEB77A
:1048B0001196CD92DC9212978DE993E282839383D5
:1048C000048315830E948D17EDB7FEB73696EDBFB2
:1048D000FEBFA496CDBFDEBFCF91DF911F910F9198
:1048E000FF90EF90DF90CF900895EF92FF920F939B
:1048F0001F93CF93DF93EC0162307105BCF1DA01B5
:1049000012968D919C91139763E872E2AE010E941A
:10491000C0108C0197FD05C03EE2E32E32E2F32E7B
:1049200004C021E3E22E22E2F22EC8010E94161DED
:10493000EDB7FEB73A97EDBFFEBF3196ADB7BEB744
:104940001196CD93DC93129725E332E222833383D1
:10495000E482F58206831783808791870E948D17F2
:10496000EDB7FEB73A96EDBFFEBF14C000D00F9270
:10497000ADB7BEB711968D939C9312978EEA93E2D2
:1049800013968D939C9314970E948D170F900F9000
:104990000F900F90DF91CF911F910F91FF90EF90AB
:1049A0000895CF92DF92EF92FF920F931F93DF93C0
:1049B000CF9300D000D0CDB7DEB76C016230710567
:1049C0000CF45DC0DA0112968D919C911397BE0193
:1049D0006F5F7F4F0E944320009709F450C0898188
:1049E0009A81BE016D5F7F4F0E9494108C0197FDEC
:1049F00005C05EE2E52E52E2F52E04C041E3E42E4E
:104A000042E2F42EC8010E94161DEDB7FEB73A9798
:104A1000EDBFFEBF3196ADB7BEB71196CD92DC9219
:104A2000129720ED33E222833383E482F5820683FA
:104A30001783808791870E948D17EDB7FEB73A964E
:104A4000EDBFFEBFCE0103960E94AE1500D000D090
:104A5000EDB7FEB73196ADB7BEB71196CD92DC92E9
:104A600012972CED33E222833383848395830E9453
:104A70008D17EDB7FEB73696EDBFFEBF14C000D060
:104A80000F92ADB7BEB71196CD92DC92129786EE1B
:104A900093E213968D939C9314970E948D170F9019
:104AA0000F900F900F902696CDBFDEBFCF91DF9174
:104AB0001F910F91FF90EF90DF90CF9008952F926C
:104AC0003F924F925F926F927F928F929F92AF929E
:104AD000BF92CF92DF92EF92FF920F931F93DF93DB
:104AE000CF93CDB7DEB72897CDBFDEBF4C017B019A
:104AF0008A01643071050CF4CEC0DA0112968D91F2
:104B00009C911397BE016F5F7F4F0E9443200097D7
:104B100009F4C1C0F5E0AF2EB12CAC0EBD1EF801FA
:104B200084819581B5010E943F14009709F4B3C0B8
:104B3000D80116968D919C911797BE016D5F7F4F9E
:104B40000E946C20009709F4A6C0B801685F7F4FEF
:104B5000C70104970E948E1B6C01009709F471C075
:104B60000E9427163C01C5010E94AE15EDB7FEB7A5
:104B70003A97EDBFFEBF3196ADB7BEB711968D9295
:104B80009C92129725E034E22283338364827582FB
:104B9000868397838B819C81808791870E948D1764
:104BA000EDB7FEB73A96EDBFFEBFEE24FF243A2CD8
:104BB0002B2CE1E24E2EE4E25E2E36C05301AE18FD
:104BC000BF08B6016E0D7F1D0B811C8189819A8102
:104BD000A501232D322D0E9442108C0197FF04C0A5
:104BE000C6010E946C512FC02DB73EB728503040EF
:104BF0002DBF3EBFEDB7FEB73196ADB7BEB711962C
:104C00008D929C9212974282538284839583A81A34
:104C1000B90AA682B7820E948D17E00EF11EEDB789
:104C2000FEB73896EDBFFEBFE614F7043CF2C601AE
:104C30000E946C5100E010E07EE2E72E72E2F72E57
:104C400006C00DEF1FEF61E3E62E62E2F62EC8010B
:104C50000E94161D2DB73EB72A5030402DBF3EBFD3
:104C6000EDB7FEB73196ADB7BEB711968D929C9257
:104C7000129725E332E222833383E482F5820683AE
:104C80001783808791870E948D17EDB7FEB73A96FC
:104C9000EDBFFEBF14C000D00F92ADB7BEB71196E6
:104CA0008D929C92129786E394E213968D939C9337
:104CB00014970E948D170F900F900F900F902896C9
:104CC000CDBFDEBFCF91DF911F910F91FF90EF908D
:104CD000DF90CF90BF90AF909F908F907F906F901C
:104CE0005F904F903F902F9008954F925F926F92F8
:104CF0007F928F929F92AF92BF92CF92DF92EF926C
:104D0000FF920F931F93DF93CF930F920F92CDB724
:104D1000DEB74C017B018A01633071050CF4A1C040
:104D2000DA0112968D919C911397BE016F5F7F4FB0
:104D30000E944320009709F494C0B8016C5F7F4F34
:104D4000C70102970E948E1B6C01009709F45FC097
:104D50000E9427165C0100D000D0EDB7FEB7319657
:104D6000ADB7BEB711968D929C92129786E694E2EB
:104D700082839383A482B5820E948D17EDB7FEB71C
:104D80003696EDBFFEBF00E010E0B1E24B2EB4E27C
:104D90005B2E32C03501601A710AB601600F711FB7
:104DA00089819A81A3010E9409107C0197FF04C0A8
:104DB000C6010E946C512FC02DB73EB7285030401D
:104DC0002DBF3EBFEDB7FEB73196ADB7BEB711965A
:104DD0008D929C9212974282538284839583681AA3
:104DE000790A668277820E948D170E0D1F1DEDB71E
:104DF000FEB73896EDBFFEBF0A151B055CF2C60173
:104E00000E946C51EE24FF240EE212E206C0ADEFC8
:104E1000EA2EAFEFFA2E01E312E2C7010E94161D3F
:104E20002DB73EB72A5030402DBF3EBFEDB7FEB77D
:104E30003196ADB7BEB711968D929C92129725E32D
:104E400032E22283338304831583E682F7828087EC
:104E500091870E948D17EDB7FEB73A96EDBFFEBF62
:104E600014C000D00F92ADB7BEB711968D929C9230
:104E7000129789E794E213968D939C9314970E945E
:104E80008D170F900F900F900F900F900F90CF9164
:104E9000DF911F910F91FF90EF90DF90CF90BF9027
:104EA000AF909F908F907F906F905F904F900895FC
:104EB000CF92DF92EF92FF920F931F93DF93CF93E6
:104EC0000F920F92CDB7DEB76C0162307105ECF135
:104ED000DA0112968D919C911397BE016F5F7F4FFF
:104EE0000E944320009789F189819A810E94060FD0
:104EF0008C0197FD05C09EE2E92E92E2F92E04C0D6
:104F000081E3E82E82E2F82EC8010E94161DEDB75B
:104F1000FEB73A97EDBFFEBF3196ADB7BEB711965B
:104F2000CD92DC92129725E332E222833383E4822E
:104F3000F58206831783808791870E948D17EDB7CE
:104F4000FEB73A96EDBFFEBF14C000D00F92ADB7CA
:104F5000BEB71196CD92DC9212978BE994E213962C
:104F60008D939C9314970E948D170F900F900F9024
:104F70000F900F900F90CF91DF911F910F91FF90A5
:104F8000EF90DF90CF900895CF92DF92EF92FF9253
:104F90000F931F93DF93CF93CDB7DEB72897CDBF85
:104FA000DEBF6C018A01643071050CF45BC0DA016C
:104FB00012968D919C911397BE016F5F7F4F0E9457
:104FC0004320009709F44EC045E0E42EF12CEC0E8E
:104FD000FD1EF80184819581B7010E943F1400975E
:104FE00009F440C0D80116968D919C911797BE0187
:104FF0006D5F7F4F0E946C200097A1F14B815C8117
:1050000089819A81B7010E946E0E8C0197FD05C0BF
:105010003EE2E32E32E2F32E04C021E3E22E22E24E
:10502000F22EC8010E94161DEDB7FEB73A97EDBFEC
:10503000FEBF3196ADB7BEB71196CD92DC921297F6
:1050400025E332E222833383E482F58206831783E9
:10505000808791870E948D17EDB7FEB73A96EDBF16
:10506000FEBF14C000D00F92ADB7BEB71196CD925F
:10507000DC92129783EB94E213968D939C93149792
:105080000E948D170F900F900F900F902896CDBF14
:10509000DEBFCF91DF911F910F91FF90EF90DF90D6
:1050A000CF900895CF92DF92EF92FF920F931F93CC
:1050B000DF93CF9300D00F92CDB7DEB76C017B01A9
:1050C0008A0181E090E08B839C83623071050CF44F
:1050D00054C0DA0112968D919C911397BE016F5FB7
:1050E0007F4F0E944320009709F447C0B2E0EB16BF
:1050F000F10451F0F80184819581BE016D5F7F4F0D
:105100000E9443200097C9F16B817C8189819A813B
:105110004DED58E296010E94300E8C0197FD05C0BE
:105120006EE2E62E62E2F62E04C051E3E52E52E274
:10513000F52EC8010E94161D2DB73EB72A503040EB
:105140002DBF3EBFEDB7FEB73196ADB7BEB71196D6
:10515000CD92DC92129725E332E222833383E482FC
:10516000F58206831783808791870E948D17EDB79C
:10517000FEB73A96EDBFFEBF14C000D00F92ADB798
:10518000BEB71196CD92DC92129789ED94E21396F8
:105190008D939C9314970E948D170F900F900F90F2
:1051A0000F902496CDBFDEBFCF91DF911F910F915D
:1051B000FF90EF90DF90CF900895EF92FF920F93C2
:1051C0001F93CF93DF937C01EB0100D000D0EDB7AC
:1051D000FEB73196ADB7BEB711968C93F1828CEFC6
:1051E00094E282839383648375830E948D172DB725
:1051F0003EB72A5F3F4F2DBF3EBFCE010E94B40E87
:10520000EC011816190664F461E87FE1A7010E9419
:10521000C90DCE016EE379E2A7010E94E30D02C041
:10522000009719F40EE212E202C001E312E2CE018D
:105230000E94161DADB7BEB71A97ADBFBEBFEDB782
:10524000FEB731961196EC92F18225E332E2228389
:10525000338304831583C683D783808791870E9415
:105260008D172DB73EB7265F3F4F2DBF3EBFDF9155
:10527000CF911F910F91FF90EF900895AF92BF9241
:10528000CF92DF92EF92FF920F931F93DF93CF9312
:10529000CDB7DEB7C054D040CDBFDEBFB82EA92EEB
:1052A0006B018A014115510519F08AEA92E202C0A8
:1052B00080E295E22DB73EB72A5030402DBF3EBF69
:1052C000EDB7FEB73196ADB7BEB71196BC92A182CD
:1052D00022E335E222833383C482D5820683178397
:1052E000808791870E948D172DB73EB7265F3F4F6D
:1052F0002DBF3EBF7E010894E11CF11C18C0013493
:10530000110518F040E450E001C0A801C601B70142
:105310000E94610F9C01181619068CF7081B190BC7
:105320008B2D9A2D60E575E2A7010E9416181016C4
:1053300011062CF3C05CDF4FCDBFDEBFCF91DF91F4
:105340001F910F91FF90EF90DF90CF90BF90AF90A3
:105350000895CF92DF92EF92FF920F931F93DF9306
:10536000CF93CDB7DEB72897CDBFDEBF6C018A01E2
:10537000643071050CF45BC0DA0112968D919C913A
:105380001397BE016F5F7F4F0E944320009709F47F
:105390004EC0F5E0EF2EF12CEC0EFD1EF8018481DD
:1053A0009581B7010E943F14009709F440C0D801CD
:1053B00016968D919C911797BE016D5F7F4F0E944D
:1053C0006C200097A1F14B815C8189819A81B701A2
:1053D0000E94FD0D8C0197FD05C0EEE2EE2EE2E28B
:1053E000FE2E04C071E3E72E72E2F72EC8010E9480
:1053F000161DEDB7FEB73A97EDBFFEBF3196ADB7BC
:10540000BEB71196CD92DC92129725E332E2228349
:105410003383E482F58206831783808791870E9415
:105420008D17EDB7FEB73A96EDBFFEBF14C000D0A2
:105430000F92ADB7BEB71196CD92DC92129783E56D
:1054400095E213968D939C9314970E948D170F905D
:105450000F900F900F902896CDBFDEBFCF91DF91B8
:105460001F910F91FF90EF90DF90CF900895AF9232
:10547000BF92CF92DF92EF92FF920F931F93DF9331
:10548000CF930F920F92CDB7DEB76C015B018A010B
:1054900019821A82623071050CF479C0DA01129611
:1054A0008D919C91139766E775E20E9436160097DE
:1054B000C9F0F801828193816DE775E20E9436168A
:1054C000009799F0D80112968D919C91139763E8FB
:1054D00075E20E943616009709F059C092E0E92E55
:1054E000F12C06C0EE24FF2403C081E0E82EF12C4D
:1054F000B2E0AB16B10459F0F80184819581BE0188
:105500006F5F7F4F0E944320009709F440C069817C
:105510007A81C7010E94720D8C0161E87FE1A601CA
:105520000E94C90DC8016EE379E2A6010E94E30D55
:1055300017FD05C0BEE2EB2EB2E2FB2E04C0A1E3D4
:10554000EA2EA2E2FA2EC8010E94161D2DB73EB720
:105550002A5030402DBF3EBFEDB7FEB73196ADB7F4
:10556000BEB71196CD92DC92129725E332E22283E8
:105570003383E482F58206831783808791870E94B4
:105580008D17EDB7FEB73A96EDBFFEBF14C000D041
:105590000F92ADB7BEB71196CD92DC92129787E805
:1055A00095E213968D939C9314970E948D170F90FC
:1055B0000F900F900F900F900F90CF91DF911F9150
:1055C0000F91FF90EF90DF90CF90BF90AF90089534
:1055D000CF92DF92EF92FF920F931F93DF93CF93BF
:1055E0000F920F92CDB7DEB76C0162307105ECF10E
:1055F000DA0112968D919C911397BE016F5F7F4FD8
:105600000E944320009789F189819A810E94EF0CC2
:105610008C0197FD05C03EE2E32E32E2F32E04C07A
:1056200021E3E22E22E2F22EC8010E94161DEDB700
:10563000FEB73A97EDBFFEBF3196ADB7BEB7119634
:10564000CD92DC92129725E332E222833383E48207
:10565000F58206831783808791870E948D17EDB7A7
:10566000FEB73A96EDBFFEBF14C000D00F92ADB7A3
:10567000BEB71196CD92DC92129785EB95E2139608
:105680008D939C9314970E948D170F900F900F90FD
:105690000F900F900F90CF91DF911F910F91FF907E
:1056A000EF90DF90CF9008950F931F93DF93CF93E8
:1056B0000F920F92CDB7DEB78C01CE0101960E94FA
:1056C000D30C97FD03C02EE232E202C021E332E2A6
:1056D0004DB75EB74A5050404DBF5EBFEDB7FEB705
:1056E0003196ADB7BEB711960D931C9312974EEC41
:1056F00055E242835383248335838683978389814C
:105700009A81808791870E948D174DB75EB7465F5B
:105710005F4F4DBF5EBF0F900F90CF91DF911F91F4
:105720000F910895CF92DF92EF92FF920F931F9304
:10573000DF93CF930F920F92CDB7DEB76C0162303B
:105740007105ECF1DA0112968D919C911397BE01CF
:105750006F5F7F4F0E944320009789F189819A8172
:105760000E94C30C8C0197FD05C05EE2E52E52E25B
:10577000F52E04C041E3E42E42E2F42EC8010E945B
:10578000161DEDB7FEB73A97EDBFFEBF3196ADB728
:10579000BEB71196CD92DC92129725E332E22283B6
:1057A0003383E482F58206831783808791870E9482
:1057B0008D17EDB7FEB73A96EDBFFEBF14C000D00F
:1057C0000F92ADB7BEB71196CD92DC92129783EED1
:1057D00095E213968D939C9314970E948D170F90CA
:1057E0000F900F900F900F900F90CF91DF911F911E
:1057F0000F91FF90EF90DF90CF900895CF92DF92BE
:10580000EF92FF920F931F93DF93CF93CDB7DEB745
:105810006097CDBFDEBF6C017B018A018091E930CA
:105820009091EA30A091EB30B091EC308D839E8363
:10583000AF83B88789879A87AB87BC878D879E8718
:10584000AF87B88B623071050CF478C0DA0112961C
:105850008D919C911397BE016F5F7F4F0E943F1403
:10586000009709F46BC0B2E0EB16F10451F1F801B6
:1058700084819581BE016B5F7F4F0E943F1400972A
:1058800009F45CC0F3E0EF16F104D9F0D8011696E4
:105890008D919C911797BE01675F7F4F0E943F14C7
:1058A000009709F44BC0B4E0EB16F10451F0F80195
:1058B00080859185BE01635F7F4F0E943F140097F2
:1058C000E9F1CE010196BE016B5F7F4FAE01475FEC
:1058D0005F4F9E01235F3F4F0E94A50C8C0197FDF7
:1058E00005C07EE2E72E72E2F72E04C061E3E62EE9
:1058F00062E2F62EC8010E94161D2DB73EB72A504F
:1059000030402DBF3EBFEDB7FEB73196ADB7BEB745
:105910001196CD92DC92129725E332E222833383F3
:10592000E482F58206831783808791870E948D1712
:10593000EDB7FEB73A96EDBFFEBF14C000D00F9290
:10594000ADB7BEB71196CD92DC9212978BEF95E270
:1059500013968D939C9314970E948D170F900F9020
:105960000F900F906096CDBFDEBFCF91DF911F915A
:105970000F91FF90EF90DF90CF9008958F929F92BC
:10598000AF92BF92CF92DF92EF92FF920F931F934D
:10599000DF93CF93CDB7DEB7CC54D040CDBFDEBFC1
:1059A0004C01E2E2EE2EF12CEC0EFD1EC7010E942E
:1059B0002D0D5C018E010E5B1F4FD8014C916E01C5
:1059C0000894C11CD11CC601B70150E00E941E16EC
:1059D000F8018081F601E80FF11D1082B7FC03C0C9
:1059E0008EE292E202C081E392E22DB73EB72850E8
:1059F00030402DBF3EBFEDB7FEB73196ADB7BEB755
:105A000011968D929C9212972AE236E2228333837A
:105A100084839583A682B7820E948D17EDB7FEB767
:105A20003896EDBFFEBFFE01EE5BFF4F80818823FD
:105A300019F0CE01019602C086E296E22DB73EB77C
:105A4000265130402DBF3EBFEDB7FEB73196ADB702
:105A5000BEB711968D929C92129721E336E2228373
:105A6000338384839583DE01AD5BBF4F8C91868346
:105A70001782DE01AC5BBF4F8C9180871186DE01FF
:105A8000AB5BBF4F8C9182871386DE01AA5BBF4F51
:105A90008C9184871586DE01A95BBF4F8C91868728
:105AA0001786DE01A85BBF4F8C91808B118ADE01C7
:105AB000A75BBF4F8D919C91828B938BDE01A55B81
:105AC000BF4F8D919C91848B958B0E948D17EDB764
:105AD000FEB77696EDBFFEBFC45BDF4FCDBFDEBF26
:105AE000CF91DF911F910F91FF90EF90DF90CF90BA
:105AF000BF90AF909F908F9008950F931F93CF9377
:105B0000DF93EC018B010E942716482FF80180A338
:105B1000C801BE0150E00E941E1681E090E0DF91B6
:105B2000CF911F910F9108950F931F93DF93CF9300
:105B300000D000D0CDB7DEB78C01CE0101960E9417
:105B4000080D97FD03C02EE232E202C021E332E2EB
:105B50004DB75EB7445150404DBF5EBFEDB7FEB785
:105B60003196ADB7BEB711960D931C93129745E6CB
:105B700056E24283538324833583868397838981C6
:105B8000808711868A81828713868B818487158618
:105B90008C81868717868D81808B118A8E81828B7E
:105BA000138A0E948D174DB75EB74C5E5F4F4DBF95
:105BB0005EBF2696CDBFDEBFCF91DF911F910F91C3
:105BC0000895CF92DF92EF92FF920F931F93DF938E
:105BD000CF930F920F92CDB7DEB76C016230710593
:105BE000E4F1DA0112968D919C911397BE016F5FDB
:105BF0007F4F0E944320009781F189810E94071303
:105C00008C0197FD05C0AEE2EA2EA2E2FA2E04C096
:105C1000F1E3EF2EF2E2FF2EC8010E94161DEDB750
:105C2000FEB73A97EDBFFEBF3196ADB7BEB711963E
:105C3000CD92DC92129725E332E222833383E48211
:105C4000F58206831783808791870E948D17EDB7B1
:105C5000FEB73A96EDBFFEBF14C000D00F92ADB7AD
:105C6000BEB71196CD92DC9212978DE896E213960C
:105C70008D939C9314970E948D170F900F900F9007
:105C80000F900F900F90CF91DF911F910F91FF9088
:105C9000EF90DF90CF900895AF92BF92CF92DF92B6
:105CA000EF92FF920F931F93DF93CF93CDB7DEB7A1
:105CB0006097CDBFDEBF5C018A016630710509F0D7
:105CC000AFC0DA0112968D919C911397BE016F5F60
:105CD0007F4F0E944320009709F4A2C0F8018481FD
:105CE0009581BE016B5F7F4F0E94A11F61157105F9
:105CF0008105910509F494C0D80116968D919C9167
:105D00001797BE01675F7F4F0E94A11F6115710544
:105D10008105910509F484C0F80180859185BE0153
:105D20006D5F7F4F0E944320009709F479C0D8012E
:105D30001A968D919C911B97BE01635F7F4F0E94C5
:105D4000A11F611571058105910509F469C0EDB7C1
:105D5000FEB73E97EDBFFEBF3196ADB7BEB7119609
:105D6000AD92BC9212978CEA96E2828393838981EA
:105D70009A81848395838D819E818683978389858B
:105D80009A85808791878B819C81828793878D8577
:105D90009E85848795870E948D17EDB7FEB73E9646
:105DA000EDBFFEBF4D815E816F81788509851A85C3
:105DB0002B853C85CD84DE848981EB800E942B136A
:105DC0008C0197FD05C08EE2E82E82E2F82E04C019
:105DD000B1E3EB2EB2E2FB2EC8010E94161D2DB7D7
:105DE0003EB72A5030402DBF3EBFEDB7FEB73196CB
:105DF000ADB7BEB71196AD92BC92129725E332E2D1
:105E000022833383E482F582068317838087918718
:105E10000E948D17EDB7FEB73A96EDBFFEBF1EC0CC
:105E200000D00F92ADB7BEB71196AD92BC9212974B
:105E30008DEB96E213968D939C9314970E948D1789
:105E4000EDB7FEB7A182B28281EF96E2838394839D
:105E50000E948D170F900F900F900F906096CDBFFE
:105E6000DEBFCF91DF911F910F91FF90EF90DF90F8
:105E7000CF90BF90AF900895CF92DF92EF92FF92B4
:105E80000F931F93DF93CF930F920F92CDB7DEB78F
:105E90006C0162307105ECF1DA0112968D919C91E2
:105EA0001397BE016F5F7F4F0E944320009789F1D7
:105EB00089819A810E9417138C0197FD05C02EE2FB
:105EC000E22E22E2F22E04C091E3E92E92E2F92EB4
:105ED000C8010E94161DEDB7FEB73A97EDBFFEBF91
:105EE0003196ADB7BEB71196CD92DC92129725E3ED
:105EF00032E222833383E482F5820683178380872C
:105F000091870E948D17EDB7FEB73A96EDBFFEBFA1
:105F100014C000D00F92ADB7BEB71196CD92DC92EF
:105F200012978DE297E213968D939C9314970E949B
:105F30008D170F900F900F900F900F900F90CF91A3
:105F4000DF911F910F91FF90EF90DF90CF90089518
:105F50000F931F93DF93CF930F92CDB7DEB78C01D2
:105F6000CE0101960E94E81297FD03C04EE252E274
:105F700002C041E352E22981222319F423E437E2EB
:105F800002C027E437E26DB77EB76A5070406DBF3C
:105F90007EBFEDB7FEB73196ADB7BEB711960D9384
:105FA0001C93129765E372E2628373834483558383
:105FB00086839783208731870E948D176DB77EB7C0
:105FC000665F7F4F6DBF7EBF0F90CF91DF911F91B6
:105FD0000F910895EF92FF920F931F93CF93DF934A
:105FE0008C01EA01623071050CF445C08A819B8105
:105FF00063E477E20E943616009751F08A819B8114
:1060000067E477E20E9436160097A9F581E001C0A7
:1060100080E00E94D812EC0197FD05C04EE2E42E0C
:1060200042E2F42E04C031E3E32E32E2F32ECE013D
:106030000E94161D2DB73EB72A5030402DBF3EBFDF
:10604000EDB7FEB73196ADB7BEB711960D931C9361
:10605000129725E332E222833383E482F582C683FA
:10606000D783808791870E948D17EDB7FEB73A9648
:10607000EDBFFEBF14C000D00F92ADB7BEB71196F2
:106080000D931C9312978AE497E213968D939C9339
:1060900014970E948D170F900F900F900F90DF9123
:1060A000CF911F910F91FF90EF900895EF92FF9283
:1060B0000F931F93CF93DF937C010E94970CEC0109
:1060C00097FD03C00EE212E202C001E312E2CE012C
:1060D0000E94161D2DB73EB72A5030402DBF3EBF3F
:1060E000EDB7FEB73196ADB7BEB71196ED92FC9203
:1060F000129725E332E22283338304831583C68318
:10610000D783808791870E948D172DB73EB7265F72
:106110003F4F2DBF3EBFDF91CF911F910F91FF9059
:10612000EF900895AF92BF92CF92DF92EF92FF92DD
:106130000F931F93DF93CF93CDB7DEB7A197CDBF5A
:10614000DEBF5C016B018A017E010894E11CF11C39
:10615000C70160E070E041E250E00E94211624E0B7
:10616000C216D104A4F1D80112968D919C91139777
:10617000B7010E947D2D009709F487C0F801E680E1
:10618000F780C70165E677E20E943616009791F026
:10619000C7016AE677E20E943616009771F0C701E0
:1061A0006EE677E20E943616009709F06EC041E075
:1061B00050E005C043E050E002C042E050E0D801AA
:1061C00014966D917C911597CE0101962CC0B3E089
:1061D000CB16D10481F4F80182819381B7010E942A
:1061E0007D2D009709F451C0D80114966D917C91D2
:1061F0001597C70116C0B2E0CB16D10451F4F801CF
:1062000082819381B7010E947D2D0097F1F1C70132
:1062100006C0F1E0CF16D104C1F580E090E060E067
:1062200070E040E050E00E943B0C8C0197FD05C0FF
:106230006EE2E62E62E2F62E04C051E3E52E52E253
:10624000F52EC8010E94161D2DB73EB72A503040CA
:106250002DBF3EBFEDB7FEB73196ADB7BEB71196B5
:10626000AD92BC92129725E332E222833383E4821B
:10627000F58206831783808791870E948D17EDB77B
:10628000FEB73A96EDBFFEBF14C000D00F92ADB777
:10629000BEB71196AD92BC92129782E797E2139621
:1062A0008D939C9314970E948D170F900F900F90D1
:1062B0000F90A196CDBFDEBFCF91DF911F910F91BF
:1062C000FF90EF90DF90CF90BF90AF9008958F92A6
:1062D0009F92AF92BF92CF92DF92EF92FF920F9375
:1062E0001F93DF93CF9300D00F92CDB7DEB74C0151
:1062F0006A0119821A821B821C8263307105A4F024
:10630000DA0112968D919C911397BE016F5F7F4FBA
:106310000E944320009709F46AC0F60184819581A8
:10632000BE016D5F7F4F0CC06230710509F05FC028
:10633000DA0112968D919C911397BE016F5F7F4F8A
:106340000E944320009709F452C069817A8188270E
:1063500077FD8095982F4B810E941E0B5C01009762
:1063600001F584E690E00E94F44549815A81662750
:1063700057FD6095762FCB80DC8080917E319091A7
:106380007F3128E030E000E010E0E1E0EE2EF12C7B
:106390000E94624497FD40C084E690E00E94F4456C
:1063A00002C097FD03C00EE212E202C001E312E256
:1063B000C5010E94161DEDB7FEB73A97EDBFFEBFAF
:1063C0003196ADB7BEB711968D929C92129725E388
:1063D00032E22283338304831583A682B7828087C7
:1063E00091870E948D17EDB7FEB73A962BC000D06B
:1063F0000F92ADB7BEB711968D929C9212978EE90F
:1064000097E213968D939C9314970E948D170F908B
:106410000F900F900F9018C000D000D0EDB7FEB7CE
:106420003196ADB7BEB711968D929C92129728EC1B
:1064300037E222833383848395830E948D17EDB7DF
:10644000FEB73696EDBFFEBF2496CDBFDEBFCF911F
:10645000DF911F910F91FF90EF90DF90CF90BF9051
:10646000AF909F908F900895EF92FF920F931F939C
:10647000CF93DF937C010E94460BEC0197FD03C094
:106480000EE212E202C001E312E2CE010E94161DEA
:106490002DB73EB72A5030402DBF3EBFEDB7FEB7F7
:1064A0003196ADB7BEB71196ED92FC92129725E3E7
:1064B00032E22283338304831583C683D7838087A4
:1064C00091870E948D172DB73EB7265F3F4F2DBF96
:1064D0003EBFDF91CF911F910F91FF90EF900895F4
:1064E000CF93DF93EC0188819981009721F00E947E
:1064F000060F18821982DF91CF9108950F931F9391
:10650000CF93DF938C01FC0182819381009721F06E
:10651000C80102960E947032F801808191810E9428
:10652000B40EEC0197FD0EC067EA72E3A8010E9469
:10653000C90DCE0160EC72E3A8010E94E30DF801E1
:10654000C283D383DF91CF911F910F910895DF9381
:10655000CF9300D00F92CDB7DEB74115510539F07A
:10656000CB01BE016F5F7F4F0E94941003C0029663
:106570000E9470322496CDBFDEBFCF91DF91089587
:10658000AF92BF92CF92DF92EF92FF920F931F9341
:10659000CF93DF935B016A01E82EE7017E01F92EBC
:1065A000E7014115510509F453C086E0E82EF12CAE
:1065B000EC0EFD1ECB01B70140E850E00E94610FD8
:1065C0008C01A601481B590BC50160E070E00E94D8
:1065D000610F17FD41C08A819B810097E9F1FE019F
:1065E000E00FF11F1582C7016FED7BE20E94761666
:1065F000009791F1C70162EE7BE244E050E00E9417
:106600003316009729F5FE013A96CF0121912C30DF
:10661000E1F32A30D1F32D30C1F32930B1F32B301F
:10662000A1F3203291F3E82FF92FDF0121912C30D3
:1066300051F02A3041F02D3031F0293021F02B304B
:1066400011F0203291F71C926A817B810E94944064
:10665000CE0102960E947032DF91CF911F910F916F
:10666000FF90EF90DF90CF90BF90AF900895CF92C2
:10667000DF92EF92FF920F931F93CF93DF937C01F2
:1066800086E890E00E941216C82EE6016E01D92E0F
:10669000E6018601209739F180E090E060E070E04B
:1066A0000E94720D8883998397FD12C069EE70E392
:1066B000A7010E94FD0D009759F48881998161E03E
:1066C00070E04EE752E396010E94300E009759F0B9
:1066D00088819981009711F00E94060FCE010E94D7
:1066E0001B1600E010E0C801DF91CF911F910F91C0
:1066F000FF90EF90DF90CF900895CF93DF93EC0160
:1067000002960E94703288819981009711F00E9450
:10671000060FCE010E941B16DF91CF910895EF92D4
:10672000FF920F931F93CF93DF938C01CB01EA016C
:1067300079010E94AE1500D000D0EDB7FEB73196BA
:10674000ADB7BEB711960C93118327EE3BE22283BF
:106750003383848395830E948D170F920F92EDB738
:10676000FEB73196ADB7BEB711960C93118384E096
:106770009CE282839383C483D583E682F7820E945E
:106780008D178DB79EB708968DBF9EBFDF91CF91B5
:106790001F910F91FF90EF900895CF92DF92EF92AB
:1067A000FF920F931F93CF93DF93D82EC92E7B01B7
:1067B000CA01E90101151105A1F40E94AE152DB71A
:1067C0003EB72A5030402DBF3EBFEDB7FEB73196E1
:1067D000ADB7BEB71196DC921197C1822AE23CE2B6
:1067E00012C003301105F1F40E94AE15ADB7BEB76B
:1067F0001A97ADBFBEBFEDB7FEB731961196DC92CA
:10680000C1822AE43CE222833383E482F5828683D8
:106810009783C087D1870E948D172DB73EB7265F1B
:106820003F4F1FC00E94AE15ADB7BEB71C97ADBF9E
:10683000BEBFEDB7FEB731961196DC92C18227E854
:106840003CE222833383E482F58286839783C08788
:10685000D187028713870E948D172DB73EB7245F1B
:106860003F4F2DBF3EBFDF91CF911F910F91FF9002
:10687000EF90DF90CF900895CF93DF93EC01888D58
:10688000998D1816190614F40E94060F8A8D9B8D97
:10689000009711F00E948A1D8C819D810E941B1619
:1068A000CE010E941B16DF91CF910895CF92DF9207
:1068B000EF92FF920F931F93CF93DF93E62EE701A2
:1068C0007E01F72EE7010C811D81288939898A898B
:1068D0009B892817390781F4EA85FB85309741F0B9
:1068E0004C895D892E893F898C859D85B7011995D5
:1068F000CE010E943C347DC0EE80FF80E8E0F0E0F5
:10690000EE0EFF1E88E0F80180831182128213824E
:106910008E859F850E94F913F80184839583888969
:1069200099890E94F913F80186839783B70180E063
:1069300090E0DC010FC0D080CC24218130E02C29F4
:106940003D29329640E050E0820F931FA41FB51FEF
:10695000625070406230710570F797013695279547
:10696000F901EE0FFF1FE00FF11F220F331FE21698
:10697000F30641F0308120E040E050E0820F931FA9
:10698000A41FB51F9D0144275527A070B070820F2A
:10699000931FA41FB51FA0FF09C09D0144275527C1
:1069A000A070B070820F931FA41FB51F0E94F9132F
:1069B00080959095F80182839383888D998DB80195
:1069C000A7019E0100E010E00E9442108E159F0575
:1069D00029F48C899D8901968C8B9D8B8A8D9B8D4A
:1069E00068EE73E00E94CE1D888999890196888B94
:1069F000998BDF91CF911F910F91FF90EF90DF90D6
:106A0000CF9008958F929F92AF92BF92CF92DF92D4
:106A1000EF92FF920F931F93CF93DF93C82EA92E6F
:106A20007B018A01CA010E940F16882EE4014E01E3
:106A3000992EE4012097C9F1C701B401A8010E9471
:106A4000610F7C018017910781F58C31910568F108
:106A50000C2D1A2D74E1C72ED12CC80CD91CF601AF
:106A6000848195810E94FD13F80126853785821760
:106A70009307D9F4868997890196868B978B8084B2
:106A800091848114910489F0A484B584F6018681EF
:106A900097810E94FD139C01AE01445F5F4F0C89FA
:106AA000C501B70110E0F4011995CE010E941B1633
:106AB000DF91CF911F910F91FF90EF90DF90CF90DA
:106AC000BF90AF909F908F9008952F923F924F92DA
:106AD0005F926F927F928F929F92AF92BF92CF926E
:106AE000DF92EF92FF920F931F93DF93CF930F925A
:106AF0000F92CDB7DEB75C013B01490168018CE123
:106B000090E049835A830E9412161C0149815A81E0
:106B1000009709F442C08A01C80108960E94121623
:106B2000F101848395830097A9F182E090E061E010
:106B300070E00E94720DF101808F918F1816190676
:106B40004CF562E075E3A1010E94E30DF50180813F
:106B50009181A281B381F10180839183A283B38368
:106B6000628A738A068317831686178680869186C3
:106B7000C286D386E486F58680E090E060E070E02F
:106B800046E554E391010E943C1DF101828F938FF1
:106B9000009731F4C1010E943C342DEF3FEF02C059
:106BA00020E030E0C9010F900F90CF91DF911F914D
:106BB0000F91FF90EF90DF90CF90BF90AF909F909C
:106BC0008F907F906F905F904F903F902F9008959F
:106BD0002F923F924F925F926F927F928F929F92ED
:106BE000AF92BF92CF92DF92EF92FF920F931F93DB
:106BF000DF93CF9300D00F92CDB7DEB72C015B01AE
:106C00006A018091E9309091EA30A091EB30B09127
:106C1000EC3089839A83AB83BC8331E0E32EF12C83
:106C200020E2622E712C93E0892E912C1E01089493
:106C3000211C311C47C08701000F111F0C0D1D1DA9
:106C4000D8018D919C9166EB7CE20E9436160097EC
:106C500091F40894E11CF11CEA14FB040CF076C0DA
:106C6000F701EE0FFF1FEC0DFD1D808191810E9449
:106C70000B544C0124C0F8018081918169EB7CE2C6
:106C80000E943616009791F40894E11CF11CEA1456
:106C9000FB040CF05BC0F701EE0FFF1FEC0DFD1DB8
:106CA000808191810E940B543C0109C0D8018D91D3
:106CB0009C91B1010E943F14009709F447C00894C9
:106CC000E11CF11CEA14FB040CF4B5CF89819A8114
:106CD000AB81BC810097A105B105C1F1CE01019640
:106CE000B401A3012DEC33E30FE813E372010E941A
:106CF00065358C0197FD05C0FFEAEF2EFCE2FF2E03
:106D000004C0E2EBEE2EECE2FE2EC8010E94161D3E
:106D1000EDB7FEB73A97EDBFFEBF3196ADB7BEB740
:106D200011964D925C9212972CEB3CE222833383B6
:106D3000E482F58206831783808791870E948D17EE
:106D4000EDB7FEB73A96EDBFFEBF14C000D00F926C
:106D5000ADB7BEB711964D925C92129789EC9CE24A
:106D600013968D939C9314970E948D170F900F90FC
:106D70000F900F902496CDBFDEBFCF91DF911F9172
:106D80000F91FF90EF90DF90CF90BF90AF909F90CA
:106D90008F907F906F905F904F903F902F900895CD
:106DA000AF92BF92CF92DF92EF92FF920F931F9319
:106DB000CF93DF93B82EA92EEB016A0178018901E8
:106DC00000D00F92EDB7FEB73196ADB7BEB71196B2
:106DD0008C9391838AEF9CE2828393830E948D1728
:106DE0000F900F900F900F902097E1F0CE010E942E
:106DF000161DEDB7FEB73897EDBFFEBF3196ADB7A4
:106E0000BEB71196BC92A1822DEF3CE22283338360
:106E1000C483D583868397830E948D17EDB7FEB711
:106E2000389645C0E114F1040105110559F12DB75B
:106E30003EB72E5030402DBF3EBFCDB7DEB72196B6
:106E4000ADB7BEB71196BC92A98280E19DE28A835C
:106E50009B83CC82DD82EE82FF8208871987B60190
:106E6000882777FD8095982FA80197010E945C5094
:106E70002A873B874C875D870E948D17EDB7FEB749
:106E80003E9615C000D000D0EDB7FEB73196ADB735
:106E9000BEB71196BC92A18282E49DE28283938365
:106EA000C482D5820E948D17EDB7FEB73696EDBF2E
:106EB000FEBFDF91CF911F910F91FF90EF90DF9078
:106EC000CF90BF90AF9008950F931F93CF93DF9310
:106ED0008C01EB0100D00F92EDB7FEB73196ADB744
:106EE000BEB711968C93118388E69DE282839383CB
:106EF0000E948D170F900F900F900F901C161D067B
:106F0000DCF4CE0160E570E00E9449500097A1F4E6
:106F100000D00F92EDB7FEB73196ADB7BEB7119660
:106F20000C9311838AEF9CE2828393830E948D17D6
:106F30000F900F900F900F90DF91CF911F910F91B5
:106F40000895AF92BF92CF92DF92EF92FF920F938C
:106F50001F93CF93DF93EC01B62EA72E88899989D2
:106F6000009761F02C813D818E819F81289F600177
:106F7000299FD00C389FD00C112404C0CA88DB880C
:106F8000EC88FD886C857D85888599850E94AC1E7E
:106F9000EA8DFB8D309749F08C0120E030E08C8D3C
:106FA0009D8D6B2D7A2DA60119958A819B810E945A
:106FB0001B16888199810E94060F888999890097FC
:106FC00021F48E899F890E94060FCE010E941B1614
:106FD0008B2D9A2DDF91CF911F910F91FF90EF9004
:106FE000DF90CF90BF90AF900895EF92FF92CF9334
:106FF000DF93E82EE7017E01F92EE701CB010E9425
:10700000B40EBC018E8B9F8B97FF04C0C7010E94FA
:10701000A13714C060E778E3A7010E94C90D8E89EB
:107020009F8963E278E3A7010E94E30D0E94E11DBE
:10703000A0E0B0E088879987AA87BB87DF91CF91CE
:10704000FF90EF900895EF92FF92CF93DF939B0113
:10705000E82EE7017E01F92EE701888999890097DA
:10706000D1F54115510561F40E94E11DA0E0B0E0A9
:107070008C879D87AE87BF87C70160E070E00BC03B
:107080006A817B814C815D81C9010E94610FBC01D5
:1070900097FF04C0C7010E94A1371DC0AE81BF8108
:1070A0001196AE83BF83882777FD8095982F2A8914
:1070B0003B894C895D89260F371F481F591F2A8B32
:1070C0003B8B4C8B5D8BE88DF98D309721F08C8D4F
:1070D0009D8DBD011995DF91CF91FF90EF9008959F
:1070E000EF92FF920F931F93CF93DF93E82EE70168
:1070F0007E01F92EE7014115510521F4C7016CEF1E
:107100007FEF3CC00E94E11DA0E0B0E08887998736
:10711000AA87BB87EE24FF241EC06A817B81600F93
:10712000711F401B510B888199810E940910BC017D
:1071300097FD08C0080F191F4C815D8104171507C2
:1071400060F325C0CE011AC08C8D9D8DB7011995B5
:107150000894E11CF11C8E819F81E816F90618F451
:1071600000E010E0E9CF0E94E11DA0E0B0E08C87D4
:107170009D87AE87BF87CE0160E070E00E94A13797
:10718000DF91CF911F910F91FF90EF900895E88DBF
:10719000F98D3097C9F6DCCF2F923F924F925F92D4
:1071A0006F927F928F929F92AF92BF92CF92DF9217
:1071B000EF92FF920F931F93CF93DF932C013B012C
:1071C0004A0159014115510509F455C021153105F0
:1071D00009F451C06115710509F44DC08EE190E0CC
:1071E0000E941216282EE1011E01392EE10120977E
:1071F00009F444C08E829F82AC82BD82088F198FB1
:10720000EA8EFB8ECC8EDD8E81E090E0888B998BB0
:10721000C5010E940F168A839B83009721F4C10148
:107220006DEF7FEF0CC080E090E060E070E00E94C6
:10723000720DBC018883998397FF05C0CE010E941F
:10724000A1379C011DC0B201A3010E946E0EBC01BA
:1072500097FDF4CF8881998160E778E3A1010E94CE
:10726000C90D8881998163E278E3A1010E94E30D51
:107270002881398105C02EEF3FEF02C02DEF3FEF8F
:10728000C901DF91CF911F910F91FF90EF90DF9097
:10729000CF90BF90AF909F908F907F906F905F90B6
:1072A0004F903F902F9008956F927F928F929F9270
:1072B000AF92BF92CF92DF92EF92FF920F931F9304
:1072C000CF93DF934C017B015A0169018EE190E07D
:1072D0000E941216682EE3013E01792EE3012097E9
:1072E00019F480E090E010C0EC82FD82A88EB98E87
:1072F000CA8EDB8E0C8F1D8FC7010E940F168A83EA
:107300009B83009731F4C3016DEF7FEF0E94A1379B
:1073100023C080E090E060E070E00E94720DBC014C
:107320008883998397FD14C069EE70E3A4010E94DD
:10733000FD0DBC0197FD0CC08881998161E070E072
:1073400045EF57E393010E94300EBC0197FF02C046
:10735000CE01DCCF88819981DF91CF911F910F9170
:10736000FF90EF90DF90CF90BF90AF909F908F9065
:107370007F906F9008952F923F924F925F926F92FD
:107380007F928F929F92AF92BF92CF92DF92EF92B5
:10739000FF920F931F93DF93CF9300D000D0CDB710
:1073A000DEB75C014B016A018091E9309091EA30CF
:1073B000A091EB30B091EC3089839A83AB83BC838E
:1073C00022243324412C34E0532E20E034E02D835A
:1073D0003E8328E8622E23E1722E91E0E92EF12C03
:1073E00081C08701000F111F0C0D1D1DD8018D914B
:1073F0009C916AE67DE20E943616009799F4089403
:10740000E11CF11CE814F9040CF002C1F701EE0FC5
:10741000FF1FEC0DFD1D808191810E940B54682E91
:10742000792E5DC0F801808191816DE67DE20E9438
:1074300036160097A9F40894E11CF11CE814F9042D
:107440000CF0E6C0F701EE0FFF1FEC0DFD1D808173
:1074500091810E940B54282F392F2D833E833FC0EA
:10746000D8018D919C9160E77DE20E9436160097CD
:1074700099F40894E11CF11CE814F9040CF0C8C05C
:10748000F701EE0FFF1FEC0DFD1D808191810E9421
:107490000B54482E592E23C0F8018081918163E757
:1074A0007DE20E9436160097A1F0D8018D919C9143
:1074B00066E77DE20E943616009779F0F801808138
:1074C0009181BE016F5F7F4F0E943F14009739F496
:1074D0009FC0F1E02F2E312C02C0222433240894C7
:1074E000E11CF11CE814F9040CF47BCF21143104E5
:1074F000C9F089819A81AB81BC810097A105B10552
:1075000009F486C0CE010196B3014D815E819201DE
:1075100004E617E3E0EDEE2EE6E3FE2E65010E94A1
:10752000CC3809C0C301B20144E657E320ED36E38D
:1075300085010E9454398C0197FF1EC00E94161DC0
:107540002DB73EB72A5030402DBF3EBFEDB7FEB736
:107550003196ADB7BEB71196AD92BC92129729E79E
:107560003DE22283338326E83DE22483358306838C
:1075700017838087918744C02114310459F1CE01CB
:1075800001960E94AE152DB73EB72E5030402DBF4C
:107590003EBFEDB7FEB73196ADB7BEB71196AD920F
:1075A000BC9212972AE83DE2228333838483958339
:1075B000668277822D813E8120873187428653867D
:1075C000048715870E948D178DB79EB70E968DBFC5
:1075D0009EBF32C0ADB7BEB71A97ADBFBEBFEDB745
:1075E000FEB731961196AD92BC9212978BEB9DE24D
:1075F00082839383648275824682578200871187D3
:107600000E948D17EDB7FEB73A96EDBFFEBF14C0CE
:1076100000D00F92ADB7BEB71196AD92BC92129743
:1076200086EE9DE213968D939C9314970E948D177E
:107630000F900F900F900F902696CDBFDEBFCF9189
:10764000DF911F910F91FF90EF90DF90CF90BF904F
:10765000AF909F908F907F906F905F904F903F90F2
:107660002F9008950F931F93CF93DF938C01FB010D
:10767000EA01309709F5CA010E94161D2DB73EB7E1
:10768000285030402DBF3EBFEDB7FEB73196ADB7A5
:10769000BEB711960C93118327E13EE22283338318
:1076A00084839583C683D7830E948D17CDB7DEB7B9
:1076B0002896CDBFDEBF47C02DB73EB72051304022
:1076C0002DBF3EBFADB7BEB71196CDB7DEB789832C
:1076D00011961C93119787E39EE212968D939C93CB
:1076E0001397858196818459984F14968D939C9316
:1076F0001597848190E0019616968D939C93179729
:10770000838118968C93189719961C9219978281E9
:107710001A968C931A971B961C921B9781811C9624
:107720008C931C971D961C921D9780811E968C939E
:107730001E971F961C920E948D172DB73EB7205F93
:107740003F4F2DBF3EBFDF91CF911F910F91089505
:10775000CF93DF93EC018C819D811816190614F4E8
:107760000E94060F8E819F81009711F00E948A1D52
:10777000CE010E941B16DF91CF910895EF92FF92E8
:10778000CF93DF93E62EE7017E01F72EE701E88134
:10779000F981309739F08A819B8160E070E04FEE8B
:1077A0005FEF1995CE010E94A83BDF91CF91FF902A
:1077B000EF9008956F927F928F929F92AF92BF92B7
:1077C000CF92DF92EF92FF920F931F93DF93CF93AD
:1077D000CDB7DEB7E097CDBFDEBF3C018B014A01DC
:1077E0005E010894A11CB11CC50160E070E040E39B
:1077F00050E00E94211683E2898388E090E00E9495
:1078000012167C01009709F441C081E090E060E02D
:1078100070E00E94720D6C01181619067CF5F701D4
:1078200000831183828293828483958388E893E125
:1078300060E070E04EEB5BE397010E943C1DF701B6
:10784000868397830097D1F0C601B3014BE750E0E0
:107850000E946E0E8C010097A9F4C60166ED7EE3CE
:10786000A7010E94E30D97FD0CC0C601B50140E3DE
:1078700050E00E94091097FF0BC003C00DEF1FEFEF
:1078800001C08C01C7010E94A83B02C00DEF1FEF91
:10789000C801E096CDBFDEBFCF91DF911F910F9160
:1078A000FF90EF90DF90CF90BF90AF909F908F9020
:1078B0007F906F900895CF92DF92EF92FF920F9397
:1078C0001F93DF93CF9300D00F92CDB7DEB76C013B
:1078D000623071050CF440C0DA0112968D919C91D2
:1078E00013978E010F5F1F4FB8010E943F1400973E
:1078F00099F1C80162E37BE3A6010E94DA3B8C01A7
:1079000097FD05C091E6E92E9EE2F92E04C084E6BB
:10791000E82E8EE2F82EC8010E94161DEDB7FEB7C4
:107920003A97EDBFFEBF3196ADB7BEB71196CD9277
:10793000DC92129728E63EE222833383E482F582CA
:1079400006831783808791870E948D17EDB7FEB756
:107950003A96EDBFFEBF14C000D00F92ADB7BEB7D0
:107960001196CD92DC92129785E79EE213968D9345
:107970009C9314970E948D170F900F900F900F906B
:107980002496CDBFDEBFCF91DF911F910F91FF9065
:10799000EF90DF90CF9008952F923F924F925F9299
:1079A0006F927F928F929F92AF92BF92CF92DF920F
:1079B000EF92FF920F931F93DF93CF93CDB7DEB774
:1079C000C254D040CDBFDEBF6DAB7EABDE011196A1
:1079D000EDE1F1E324E301900D922150E1F7DC01A8
:1079E0006D917D918D919C9120E831E541E050E0D1
:1079F0000E945C5079018A0120E13EE040E050E0C5
:107A00000E947E50EDA9FEA922832CE330E040E0E5
:107A100050E00E947E50ADA9BEA911962C931197FB
:107A20006C93C801B7016C5F7F4F8F4F9F4F27E06A
:107A300030E040E050E00E947E50EDA9FEA9618751
:107A4000A2EBAA2EA7E0BA2EC12CD12CFEC0C801F1
:107A5000B7012DE631E040E050E00E947E506627FD
:107A600097FD639577278827992739014A01661A78
:107A7000770A880A990A6A0C7B1C8C1C9D1C6FAAC9
:107A800078AE89AE9AAE3501460108946108710856
:107A9000810891082FA838AC49AC5AAC0894210849
:107AA000310841085108C401B30124E030E040E04E
:107AB00050E00E947E502BAF3CAF4DAF5EAF23969F
:107AC0006CAF7DAF8EAF9FAF2397C401B3012CE99C
:107AD0003FEF4FEF5FEF0E947E508BAD9CADADADA1
:107AE000BEAD280F391F4A1F5B1FE20EF31E041F95
:107AF000151FC401B30120E931E040E050E00E94CD
:107B00007E506BAF7CAF8DAF9EAFE20EF31E041FB5
:107B1000151FC401B30124E630E040E050E00E94AC
:107B20007E50662797FD6395772788279927E60E6D
:107B3000F71E081F191F23968CAD9DADAEADBFADCE
:107B400023978827B7FD83959927AA27BB27E81A8B
:107B5000F90A0A0B1B0B8BAD9CADADADBEAD8827F2
:107B6000B7FD83959927AA27BB27E81AF90A0A0BBC
:107B70001B0BC201B10120E73EEF4FEF5FEF0E9408
:107B80007E50E20EF31E041F151FC201B10124E650
:107B900030E040E050E00E947E506BAF7CAF8DAF94
:107BA0009EAFE20EF31E041F151FC201B10124E0B7
:107BB00030E040E050E00E947E503B014C01E21A70
:107BC000F30A040B150BC201B10120E931E040E0DA
:107BD00050E00E947E50662797FD6395772788279F
:107BE0009927E60EF71E081F191FD401C301882725
:107BF000B7FD83959927AA27BB27E80EF91E0A1F10
:107C00001B1FC601B5016FA878AC89AC9AAC661988
:107C10007709880999092DE631E040E050E00E949B
:107C20001E50E60EF71E081F191F8BAD9CADADADA3
:107C3000BEAD8827B7FD83959927AA27BB27E81AE9
:107C4000F90A0A0B1B0B6401530117FD00CF23E057
:107C5000622E712C812C912C6A207B208C209D20FF
:107C60006114710481049104D1F4C601B50124E6C4
:107C700030E040E050E00E947E50611571058105C2
:107C8000910591F4C601B50120E931E040E050E0F2
:107C90000E947E50611571058105910529F08DE6E0
:107CA00091E0A0E0B0E004C08EE691E0A0E0B0E09A
:107CB000E816F9060A071B070CF0C9CEC5018C5659
:107CC0009740ADA9BEA915968D939C9316971796CC
:107CD000ED92FC921897611471048104910401F5EE
:107CE000C601B50124E630E040E050E00E947E503D
:107CF0006115710581059105B1F4C601B50120E951
:107D000031E040E050E00E947E5021E030E061151B
:107D100071058105910511F020E030E0C90105C031
:107D200080E090E002C081E090E02AE130E0829FB4
:107D3000F001839FF00D929FF00D1124CE0101966A
:107D4000E80FF91F78968BE090E0A0E0B0E003C068
:107D50000197A109B1093291229140E050E0E21669
:107D6000F30604071507A4F3EDA9FEA98483E21A1C
:107D7000F30A040B150BE394E38281E090E0CE5B01
:107D8000DF4FCDBFDEBFCF91DF911F910F91FF90ED
:107D9000EF90DF90CF90BF90AF909F908F907F90AB
:107DA0006F905F904F903F902F900895AF92BF9249
:107DB000CF92DF92EF92FF920F931F93DF93CF93B7
:107DC000CDB7DEB76097CDBFDEBF5B017A016C0136
:107DD0004033510580F1CA010E940F16082F192F58
:107DE0000115110569F1C501B801A7010E94610FD4
:107DF000AC018E159F0531F5D80190966D917D915E
:107E00008D919C9193974F87588B0E943C1460589A
:107E10007E478A4A934869837A838B839C83F8944C
:107E2000CE010196BE016B5F7F4F0E94CC3C7894DF
:107E30004F85588907C040EF5FEF00E010E002C0B7
:107E40004DEF5FEFD601ED91FC911197309741F026
:107E500012968D919C911397BE016B5F7F4F199580
:107E6000C8010E941B16C6010E94A83B6096CDBFA8
:107E7000DEBFCF91DF911F910F91FF90EF90DF90C8
:107E8000CF90BF90AF900895CF92DF92EF92FF9284
:107E90000F931F93CF93DF936C018B01CB010E9453
:107EA00027167C01C0E0D0E00EC0B8016C0F7D1F2A
:107EB000A7014C1B5D0BC6010E9409109C0197FD98
:107EC00007C0C80FD91FCE15DF057CF320E030E0D6
:107ED000C901DF91CF911F910F91FF90EF90DF903B
:107EE000CF9008958F929F92AF92BF92CF92DF92E0
:107EF000EF92FF920F931F93CF93DF934C015B019F
:107F00006A0180E490E00E940F167C01C0E0D0E09E
:107F10001DC086010C1B1D0B0134110514F000E47B
:107F200010E0B5016C0F7D1FC701A8010E943154FC
:107F3000C401B701A8010E9409108C0197FF04C079
:107F4000C7010E941B160AC0C80FD91FCC15DD053A
:107F500004F3C7010E941B1600E010E0C801DF9186
:107F6000CF911F910F91FF90EF90DF90CF90BF9036
:107F7000AF909F908F9008950F931F93CF93DF93AF
:107F8000EC018B01CB010E943A54AC01CE01B80147
:107F90000E94723FDF91CF911F910F910895EF9250
:107FA000FF920F931F93DF93CF93CDB7DEB76C97FC
:107FB000CDBFDEBF7C018EE49FE2A1E4B0E08B8701
:107FC0009C87AD87BE87FE013F968EE0DF011D9244
:107FD0008A95E9F7E114F10409F499C0C7016FE14A
:107FE00076E00E94BC3F9C0197FD93C08E010F5F1D
:107FF0001F4FC80160E070E040E050E020E030E05A
:108000000E94AE0C009729F4C8010E94AE158C01A5
:1080100002C00CEA1EE2C7016AE076E00E94BC3FA3
:108020009C0197FD76C0C701B8010E94443F9C01A6
:1080300097FD6FC0C7016FEE75E00E94BC3F9C01C9
:1080400097FD67C0CE0105960E94080D009789F53F
:108050008DB79EB742978DBF9EBFEDB7FEB73196E5
:10806000CE010B96ADB7BEB711968D939C93129728
:1080700082E190E08283938380EB9EE28483958308
:108080008D81868317828E81808711868F8182877A
:1080900013868885848715868985868717868A85CD
:1080A000808B118A0E9411558DB79EB742968DBF65
:1080B0009EBFC70169ED75E00E94BC3F9C0197FD22
:1080C00028C0C701BE01655F7F4F0E94443F9C01ED
:1080D00097FD1FC0C7016EEB75E00E94BC3F9C017D
:1080E00097FD17C0C70169E973E00E94BC3F9C017E
:1080F00097FD0FC0C70164EF71E00E94BC3F282FBD
:10810000392F121613062CF420E030E002C02FEFB6
:108110003FEFC9016C96CDBFDEBFCF91DF911F91BC
:108120000F91FF90EF900895EF92FF920F931F939E
:10813000DF93CF930F920F92CDB7DEB77C018B0107
:108140006EEC7EE20E943616009709F471C0C701FA
:1081500060ED7EE20E943616009709F469C0C701FF
:1081600063ED7EE24CE050E00E943316009709F088
:1081700058C000D000D0EDB7FEB73196C7010C96BD
:10818000ADB7BEB711968D939C93129780EE9EE289
:1081900082839383CE010196848395830E944955FF
:1081A0002DB73EB72A5F3F4F2DBF3EBF009709F462
:1081B0003FC089819A818330910511F18430910506
:1081C0004CF481309105B1F082309105B4F4009700
:1081D00071F02EC085309105C9F0853091059CF075
:1081E00086309105B1F08730910511F515C080E218
:1081F00090E014C081E290E011C082E290E00EC0F5
:1082000083E290E00BC084E290E008C085E290E059
:1082100005C086E290E002C087E290E00E949F45A0
:1082200007C0C7016DEE7EE20E943616009729F462
:10823000C8010E94CF3F9C0129C0C70169EF7EE2BF
:108240000E943616009781F4C8016EE57DE00E9419
:10825000BC3F9C0197FD1AC0C80169E778E045EE74
:1082600054E00E94723F08C00115110569F0C80171
:108270006AE97DE00E94BC3F282F392F12161306B1
:108280002CF420E030E002C02FEF3FEFC9010F9047
:108290000F90CF91DF911F910F91FF90EF90089574
:1082A0001F93CF93DF93EC01162FBA0180E090E08B
:1082B00026E631E040E050E00E941E5020917A31E5
:1082C00030917B3140E050E00E945C502093783147
:1082D000309379312FB7F894388181E090E002C073
:1082E000880F991F1A95E2F7880F880F832B8883D0
:1082F0002FBFDF91CF911F9108950F931F93DF93AD
:10830000CF93CDB7DEB72A97CDBFDEBFBE016C5F7E
:108310007F4F87E0FB0111928A95E9F78E010F5F8D
:108320001F4F83E0F80111928A95E9F786E088876C
:1083300081E08E8380E092E00E94224B80E092E018
:1083400060E571E40E94034C19821A828B81807F60
:1083500081608B8380E092E060E0A8010E94874BFF
:1083600082E06FE270E00E948946182F00E082E010
:108370006EE270E00E94894690E0802B912B809302
:108380007A3190937B3180E092E00E94F14A9FB76E
:10839000F894E0E0F2E08081846080839FBF2A96B9
:1083A000CDBFDEBFCF91DF911F910F910895209136
:1083B00078313091793121513140C90108956115E9
:1083C000710529F08FB7F8948093803108958091DA
:1083D00080318FBF089500D000D0EDB7FEB7319641
:1083E000ADB7BEB711968D939C93129783E09FE231
:1083F00082839383648375830E948D178DB79EB7A4
:1084000006968DBF9EBF08950F931F938C01611533
:10841000710579F500D00F92EDB7FEB73196ADB783
:10842000BEB711968C93118385E19FE2828393837B
:108430000E948D1780917C3190917D310F900F902B
:108440000F900F90009709F44CC00E947D3310925A
:108450007C3110927D3100D00F92EDB7FEB731968E
:10846000ADB7BEB711960C931197118387E29FE2C7
:1084700030C0CB010E94AE1500D000D0EDB7FEB7E2
:108480003196ADB7BEB711960C93118327E33FE247
:1084900022833383848395830E948D178DB79EB783
:1084A00006968DBF9EBF80E590E00E943733809393
:1084B0007C3190937D310097A1F000D00F92EDB701
:1084C000FEB73196ADB7BEB711960C93118387E412
:1084D0009FE2828393830E948D170F900F900F90DD
:1084E0000F901F910F9108956115710549F08EE26B
:1084F00090E00E9474468EE190E00E94F445089559
:108500008EE290E00E945F4608950E949A450E9484
:10851000E91D0895AF92BF92CF92DF92EF92FF9242
:108520000F931F93DF93CF93CDB7DEB7AB97CDBF3C
:10853000DEBF19820E94CF4580E490E065E872E4D6
:108540000E9471450E942B1D97FDACC180EA99E005
:1085500040E052EC61E070E028E030E000E010E044
:10856000E1E0EE2EF12CCC24DD240E94624497FD44
:1085700099C180E090E062EC74E440EA59E024E0C4
:1085800030E00E94101B5C01009709F48BC10E942F
:10859000251F80EA9BE040E052EC61E070E028E0BB
:1085A00030E00E94624497FD7DC180E090E061EE82
:1085B00074E448EF54E42FED31E400EA1BE00E943C
:1085C000590A97FD6FC180EA9BE080937E319093BA
:1085D0007F310E947D4184E792E4B5010E94DC0A6C
:1085E000CE0101960E94BB0ACE0102960E94E812BB
:1085F0008BEE91E4B5010E94320C84E092E4B50167
:108600000E94FF0CC5016FE97FE240E050E00E944C
:108610003917C50169EA7FE240E050E00E9439174E
:10862000C50165EE7FE240E050E00E943917C501C8
:108630006FEE7FE240E050E00E943917C50169EF1C
:108640007FE240E050E00E943917C50163E070E32B
:1086500040E050E00E943917C5016DE070E340E052
:1086600050E00E943917C50167E170E340E050E037
:108670000E943917C50161E270E340E050E00E94BA
:108680003917C5016BE770E340E050E00E943917ED
:10869000C5016BE270E340E050E00E943917C5016C
:1086A00065E370E340E050E00E943917C5016FE3D5
:1086B00070E340E050E00E943917C50169E470E3BF
:1086C00040E050E00E943917C50163E570E340E0E7
:1086D00050E00E943917C5016DE570E340E050E0BD
:1086E0000E943917C50167E670E340E050E00E9440
:1086F0003917C50161E770E340E050E00E94391787
:10870000C50165E870E340E050E00E943917C501FB
:108710006FE870E340E050E00E943917C50169E955
:1087200070E340E050E00E943917C50163EB7FE23F
:1087300040E050E00E943917C5016DEB7FE240E058
:1087400050E00E943917C50167EC7FE240E050E03D
:108750000E943917C50161ED7FE240E050E00E94C0
:108760003917C5016BED7FE240E050E00E943917F8
:10877000C5016BE87FE240E050E00E943917C50177
:1087800065E97FE240E050E00E943917C50163EAE5
:1087900070E340E050E00E943917C5016DEA70E3D4
:1087A00040E050E00E943917C50167EB70E340E0FC
:1087B00050E00E943917C50161EC70E340E050E0E1
:1087C0000E943917C50165ED70E340E050E00E945A
:1087D0003917C5016FED70E340E050E00E94391792
:1087E000C5016BEC70E340E050E00E943917C50111
:1087F00061E87FE240E050E00E9439178A818823D7
:1088000099F566E172E088EA90EC0E9401146B83AE
:108810007C838D839E8360E07FEF8FEF9FEF0E94CC
:1088200001146F83788789879A878E01055F1F4FB0
:10883000C80167E57FE20E94391687E59FE20E9442
:1088400027168BA7C80162E67FE240E050E00E9455
:108850003B0CCE010396BE01695F7F4F40E050E0C4
:1088600020E030E00E94A50C80EA99E00E941E45BD
:10887000009751F080EA99E060E070E00E94C844FF
:10888000682FC5010E942D19898180FF06C08DE2E5
:1088900090E00E944346009711F40E940B110E9441
:1088A000141EE2CF8FEF9FEFAB96CDBFDEBFCF910F
:1088B000DF911F910F91FF90EF90DF90CF90BF90CD
:1088C000AF900895AF92BF92CF92DF92EF92FF9256
:1088D0000F931F93B82EA92EC801C114D10409F01B
:1088E00045C0255030402530310528F42F5A3E4CE4
:1088F000F901108101C010E08130910539F081301B
:10890000910538F08230910589F502C0106201C0EE
:108910001063F2E0EF16F10409F418609A01AB015C
:1089200084E0220F331F441F551F8A95D1F7213051
:1089300088E4380788EE480781E0580750F460E083
:1089400078E488EE91E00E945C502150304088E14C
:1089500003C02FEF3FEF8CE1EB2DFA2D148215832E
:1089600026833783848320E030E002C026EF3FEF88
:10897000C9011F910F91FF90EF90DF90CF90BF90B2
:10898000AF900895FC01818185FFFDCF608308953C
:108990000F931F93CF93DF938C01EB010E94E11D96
:1089A000F801209731F4818187FFFDCF208130E0ED
:1089B00002C026EF3FEFC901DF91CF911F910F91C8
:1089C0000895FC0180E090E00EC0218127FFFDCFDB
:1089D0006115710511F4208105C02081DB01A80F0C
:1089E000B91F2C930196841795077CF3CA0108954B
:1089F000CF92DF92EF92FF920F931F93CF93DF936B
:108A00006C017A01062F172FC0E0D0E00AC0F801F0
:108A100061918F01772767FD7095C6010E94C2445E
:108A20002196CE15DF059CF3C701DF91CF911F91F1
:108A30000F91FF90EF90DF90CF900895FC0121817E
:108A400030E020783070C90108958530910540F4F8
:108A5000FC01EE0FFF1FEA5AFE4C2081318102C05B
:108A600020E73FE2C9010895EF92FF920F931F9311
:108A70007B018C01E0918131F0918231309709F0D6
:108A800019956091853170918631809187319091EF
:108A900088316E0D7F1D801F911F0E94BC471F9162
:108AA0000F91FF90EF9008958093833190938431DC
:108AB0009C01B901882777FD8095982F28EE33E037
:108AC00040E050E00E941E500E945C50209385318F
:108AD00030938631409387315093883180E090E025
:108AE0000895EF92FF920F931F937C016093813161
:108AF000709382310E94DA4784E395E40E94D5475F
:108B0000C7010E945445E0908531F0908631009174
:108B10008731109188310E949B476E0D7F1D801F09
:108B2000911F0E94BC4780E090E01F910F91FF9041
:108B3000EF90089580918331909184310895CF937F
:108B4000DF93EC010E944346009721F0CE010E9482
:108B5000744603C0CE010E945F46DF91CF91089515
:108B60000E945F4608950E9474460895AB01282F25
:108B700026952695269530E0205D3F4F877061E071
:108B800070E002C0660F771F8A95E2F7C90125E001
:108B9000880F991F2A95E1F70E945947089587E0A9
:108BA000E0EAF0E082830E9493460E94EA468BE26C
:108BB00060E073E00E94B6458AE260E070E00E94E7
:108BC000B64583E090E060E10E94BC4684E090E01E
:108BD00060E10E94BC4686E090E060E10E94BC46F5
:108BE000789480E090E00895282F392FC90107C0BC
:108BF000EFE3FFE13197F1F700C000000197009724
:108C0000B9F708951F93182F8A3031F480EA99E05C
:108C10006DE070E00E94C244612F772767FD709578
:108C200080EA99E00E94C2441F91089589E891E387
:108C30000895AB01282F26952695269530E0205DD6
:108C40003F4F877061E070E002C0660F771F8A9522
:108C5000E2F7C90125E0880F991F2A95E1F70E94E4
:108C60005947089580E090E0089560FF03C060E0F8
:108C700070E004C061FF04C060E071E00E9419462A
:108C800080E090E00895E82FE695E695E695F0E01F
:108C9000F09635E0EE0FFF1F3A95E1F7908587706B
:108CA00021E030E002C0220F331F8A95E2F79223C1
:108CB00021E030E011F420E030E0C9010895E82F10
:108CC000E695E695E695F0E0F09645E0EE0FFF1F9D
:108CD0004A95E1F7877021E030E002C0220F331F90
:108CE0008A95E2F725830895E82FE695E695E695BF
:108CF000F0E0F09655E0EE0FFF1F5A95E1F7877010
:108D000021E030E002C0220F331F8A95E2F726836C
:108D100008954091CA01E62FF72F8093CA018491EC
:108D20004093CA0108958FEF809370008093710083
:108D30008093720080937300809374008093750019
:108D4000809376009FB7F894809150008260809362
:108D500050009FBF8091510081FFFCCF80E490E0E4
:108D600061E00E9483489FB7F894809150008E7F05
:108D7000809350009FBF0895FC019FB7F894E0597D
:108D8000FF4F60958081862380839FBF0895FC01FB
:108D90009FB7F894E059FF4F8081862B80839FBF57
:108DA0000895AB01282F26952695269530E0205D65
:108DB0003F4F877061E070E002C0660F771F8A95B1
:108DC000E2F7C90125E0880F991F2A95E1F70E9473
:108DD0005947089580E260E073E00E94D14681E245
:108DE00060E073E00E94D14682E260E073E00E949E
:108DF000D14683E260E073E00E94D14684E260E005
:108E000073E00E94D14685E260E073E00E94D146A3
:108E100086E260E073E00E94D14687E260E073E0A2
:108E20000E94D14688E168E170E00E94D14689E164
:108E300068E170E00E94D1468AE168E170E00E943A
:108E4000D1468BE168E170E00E94D1468CE168E197
:108E500070E00E94D1468DE168E170E00E94D14649
:108E600088E768E170E00E94D14689E768E170E038
:108E70000E94D14688E067E070E00E94D1468BE016
:108E800060E071E00E94D14683E160E073E00E94FF
:108E9000D14682E160E070E00E94D1468BE160E063
:108EA00073E00E94D1468AE160E070E00E94D14602
:108EB00008950F931F93CF93DF93FC01DC0180E0B3
:108EC00090E0262F30E0E901082E02C0D595C79525
:108ED0000A94E2F7C0FF03C050964C935097019656
:108EE00011968830910579F750FF07C051FF02C0F5
:108EF000658301C06683618301C06283DF91CF9186
:108F00001F910F9108959091020481E092FD80E0FD
:108F10000895109200042091010420FDFCCFE0E0B0
:108F2000F4E0608771878093B5329093B63281E028
:108F30008093000408954FB7F8942091B532309192
:108F4000B6328091080490910904009731F4509151
:108F5000030450FF02C02F5F3F4F4FBF40E050E07F
:108F6000A90133272227A0E0B0E0282B392B4A2B78
:108F70005B2BB901CA010895E0E0F4E021E022830F
:108F8000648775876093B9327093BA328093B73231
:108F90009093B832E0E0F4E08091010480FDFACFD4
:108FA00082E0838385E0828308958093BB3290932F
:108FB000BC32089580E090E064E00E94BC4621E06D
:108FC000E0E4F0E02383E0E0F4E08FEF9FEF8287BE
:108FD0009387108611862283208308951F920F9213
:108FE0000FB60F9208B60F92112418BE8F939F935D
:108FF0008091B5329091B63201968093B5329093BC
:10900000B6329F918F910F9008BE0F900FBE0F90B8
:109010001F9018951F920F920FB60F9208B60F92DD
:1090200009B60F920BB60F92112418BE19BE1BBEC3
:10903000EF92FF920F931F932F933F934F935F9362
:109040006F937F938F939F93AF93BF93EF93FF9310
:109050006091B5327091B6324091B7325091B832CA
:1090600064177507A8F181E0E0E0F4E08283E09105
:10907000BB32F091BC32309759F100910804109145
:10908000090480E090E0CB017727662720E030E0FC
:10909000602B712B822B932B9A0140E050E0A901A9
:1090A00033272227E090B932F090BA3200E010E086
:1090B0002E293F29402B512B2617370748075907E0
:1090C00030F0CA01B9016F5F7F4F8F4F9F4F1995E5
:1090D000FF91EF91BF91AF919F918F917F916F9190
:1090E0005F914F913F912F911F910F91FF90EF90C2
:1090F0000F900BBE0F9009BE0F9008BE0F900FBED1
:109100000F901F9018951BBEFC0128ED24BF6083B3
:10911000089522E08030920771F480918D31982F6C
:109120009F5F90938D318823B9F481E090E062E0F5
:109130000E94BC46089522E08034920769F4809131
:109140008E31982F9F5F90938E31882329F482E08F
:1091500090E062E00E94BC46089522E080309207D1
:1091600069F480918D31815080938D318823B1F4E1
:1091700081E090E062E00E94C746089522E08034DA
:10918000920761F480918E31815080938E318823D3
:1091900029F482E090E062E00E94C7460895682FBB
:1091A00082E070E00E9489460895EF92FF92CF938B
:1091B000DF938130910579F08130910520F0823084
:1091C0009105F9F410C081E20E94CF48982F80E009
:1091D000EC0180E20FC085E20E94CF48982F80E02A
:1091E000EC0184E207C08FE20E94CF48982F80E014
:1091F000EC018EE20E94CF48282F30E02C2B3D2B33
:1092000002C020E030E0C901DF91CF91FF90EF90E4
:1092100008951F920F920FB60F9208B60F9209B6DB
:109220000F920BB60F92112418BE19BE1BBE2F93BE
:109230003F934F935F936F937F938F939F93AF93DE
:10924000BF93EF93FF93E0E0F2E044A155A1E091DA
:109250008931F0918A3180E092E061E01995FF91C7
:10926000EF91BF91AF919F918F917F916F915F919E
:109270004F913F912F910F900BBE0F9009BE0F9011
:1092800008BE0F900FBE0F901F9018951F920F925F
:109290000FB60F9208B60F9209B60F920BB60F9247
:1092A000112418BE19BE1BBE2F933F934F935F939B
:1092B0006F937F938F939F93AF93BF93EF93FF939E
:1092C000E8E2F2E044815581E0918931F0918A3100
:1092D00080E092E062E01995FF91EF91BF91AF912C
:1092E0009F918F917F916F915F914F913F912F91BE
:1092F0000F900BBE0F9009BE0F9008BE0F900FBECF
:109300000F901F9018951F920F920FB60F9208B6EC
:109310000F9209B60F920BB60F92112418BE19BE08
:109320001BBE2F933F934F935F936F937F938F93C6
:109330009F93AF93BF93EF93FF93E0E3F2E04481F9
:109340005581E0918931F0918A3180E092E064E0CA
:109350001995FF91EF91BF91AF919F918F917F915F
:109360006F915F914F913F912F910F900BBE0F9096
:1093700009BE0F9008BE0F900FBE0F901F9018955A
:109380001F920F920FB60F9208B60F9209B60F9266
:109390000BB60F92112418BE19BE1BBE2F933F931C
:1093A0004F935F936F937F938F939F93AF93BF93ED
:1093B000EF93FF93E8E3F2E044815581E091893136
:1093C000F0918A3180E092E068E01995FF91EF9189
:1093D000BF91AF919F918F917F916F915F914F91CD
:1093E0003F912F910F900BBE0F9009BE0F9008BEBA
:1093F0000F900FBE0F901F9018951F920F920FB6EF
:109400000F9208B60F9209B60F920BB60F92112465
:1094100018BE19BE1BBE2F933F934F935F936F935C
:109420007F938F939F93AF93BF93EF93FF93E0E46A
:10943000F2E044A155A1E0918B31F0918C3180E4B0
:1094400092E061E01995FF91EF91BF91AF919F91EB
:109450008F917F916F915F914F913F912F910F90DD
:109460000BBE0F9009BE0F9008BE0F900FBE0F905D
:109470001F9018951F920F920FB60F9208B60F9279
:1094800009B60F920BB60F92112418BE19BE1BBE5F
:109490002F933F934F935F936F937F938F939F93FC
:1094A000AF93BF93EF93FF93E8E6F2E044815581D9
:1094B000E0918B31F0918C3180E492E062E019957B
:1094C000FF91EF91BF91AF919F918F917F916F919C
:1094D0005F914F913F912F910F900BBE0F9009BE5E
:1094E0000F9008BE0F900FBE0F901F9018951F92FF
:1094F0000F920FB60F9208B60F9209B60F920BB6E5
:109500000F92112418BE19BE1BBE2F933F934F9389
:109510005F936F937F938F939F93AF93BF93EF93DB
:10952000FF93E0E7F2E044815581E0918B31F091C7
:109530008C3180E492E064E01995FF91EF91BF9146
:10954000AF919F918F917F916F915F914F913F91DB
:109550002F910F900BBE0F9009BE0F9008BE0F9079
:109560000FBE0F901F9018951F920F920FB60F927B
:1095700008B60F9209B60F920BB60F92112418BEBF
:1095800019BE1BBE2F933F934F935F936F937F93AF
:109590008F939F93AF93BF93EF93FF93E8E7F2E02E
:1095A00044815581E0918B31F0918C3180E492E0DF
:1095B00068E01995FF91EF91BF91AF919F918F91C5
:1095C0007F916F915F914F913F912F910F900BBEC3
:1095D0000F9009BE0F9008BE0F900FBE0F901F9006
:1095E00018951F93CF93DF93EC011FB7F8940E9457
:1095F00089488881816088831FBFDF91CF911F9147
:1096000008951F931FB7F894FC0120812E7F2083BB
:109610000E94AD481FBF1F91089522E0803092073D
:1096200021F481E090918D3107C022E080349207CF
:1096300039F481E090918E31992319F480E00895F6
:1096400080E00895DF92EF92FF920F931F93CF93E4
:10965000DF93EC018B0182E0C030D80719F480E081
:1096600090E006C0E2E0C034DE0721F581E090E042
:109670000E94D5487C01DFB6F894CE010E9489484B
:10968000288182E08883EC86FD86F80185819681B9
:10969000888F998F82818A8384818C8383818B8355
:1096A0008181898321708081282B2883CE010E94AB
:1096B000AD48DFBEDF91CF911F910F91FF90EF90EA
:1096C000DF900895FF920F931F93CF93DF93EC01E8
:1096D0008B01FFB6F8940E9489488881807CF8014C
:1096E0008083888D998D858396838A8182838C81FE
:1096F00084838B81838389818183CE010E94AD48DD
:10970000FFBEDF91CF911F910F91FF900895DF92DF
:10971000EF92FF920F931F93CF93DF93EC017A01A7
:10972000862F90E083709070009721F4669566957F
:1097300082E001C080E060FF8F5F8E01005E1F4FFE
:1097400090E023E0880F991F2A95E1F7080F191F71
:10975000DFB6F894CE010E948948F7018081F801B4
:109760008083F7018281F8018283F7018181F8010A
:109770008183CE010E94AD48DFBEDF91CF911F9162
:109780000F91FF90EF90DF900895DF92EF92FF929C
:109790000F931F93CF93DF93EC017A01862F90E014
:1097A00083709070009721F46695669582E001C001
:1097B00080E060FF8F5F8E01005E1F4F90E033E01E
:1097C000880F991F3A95E1F7080F191FDFB6F89433
:1097D000CE010E948948F8018081F7018083F80159
:1097E0008281F7018283F8018181F7018183CE01B3
:1097F0000E94AD48DFBEDF91CF911F910F91FF9086
:10980000EF90DF9008952FB7F89432E080309307FF
:1098100029F46093893170938A3108C032E0803432
:10982000930721F460938B3170938C312FBF08958F
:109830008091CF0187FDFCCF08951F93CF93DF93D5
:10984000C0ECD1E01A858A878BEC91E061E00E9440
:1098500083481A87DF91CF911F9108958BEC91E097
:1098600061E00E9483480895682F82E070E00E94C2
:1098700089460895CF93DF93EC0188E00E94344C31
:10988000888389E00E94344C89838AE00E94344CAA
:109890008A838BE00E94344C8B838CE00E94344C92
:1098A0008C838DE00E94344C8D8380E10E94344C87
:1098B0008E8382E10E94344C8F8383E10E94344C7A
:1098C000888784E10E94344C898785E10E94344C6A
:1098D0008A87DF91CF9108950F931F93DF93CF93E2
:1098E0000F920F92CDB7DEB789839A830E94184CEE
:1098F00000EC11E0F80112829A81918389818083C2
:1099000086E090E00E941D4CF80184810F900F903A
:10991000CF91DF911F910F910895EF92FF920F93D6
:109920001F93DF93CF9300D00F92CDB7DEB78C019A
:10993000CB014B835C8369839A830E94184C8CEC27
:10994000E82E81E0F82EF701208128602083005066
:10995000104F89819A81B8014B815C810E947754B4
:10996000F7018081877F80832496CDBFDEBFCF91B2
:10997000DF911F910F91FF90EF9008950E94184C76
:109980008091CF0181FF06C086E3E0ECF1E08287A1
:109990000E942E4C0895EF92FF921F93DF93CF9376
:1099A00000D0CDB7DEB720ECE22E21E0F22EF70199
:1099B000128569838A839B830E94BE4C0E94184C47
:1099C00023E3F701228712829B8191838A8180831E
:1099D0006981648385E382870E942E4CF701128798
:1099E0002396CDBFDEBFCF91DF911F91FF90EF9007
:1099F0000895EF92FF921F93DF93CF930F920F92F0
:109A0000CDB7DEB730ECE32E31E0F32EF70112854F
:109A10006A8389830E94184C93E3F701928712822C
:109A20001182898180836A81648312870F900F90ED
:109A3000CF91DF911F91FF90EF900895FF920F93C8
:109A40001F93CF93DF938C01C0ECD1E0F090CA015B
:109A50000E94184C83E38A871A82198280E0E0EC26
:109A6000F1E08093C001D8019D918D0194838F5FB7
:109A70008032B9F7E0ECF1E0F286DF91CF911F91EF
:109A80000F91FF900895DF93CF930F92CDB7DEB77C
:109A900089830E94184C898190E045E0880F991FC6
:109AA0004A95E1F7E0ECF1E012829183808385E34F
:109AB00090E00E941D4C0F90CF91DF910895CF92BE
:109AC000DF92EF92FF920F931F93CF93DF937C016E
:109AD0006B01EA0126C0C7018F7190700097B1F445
:109AE000C032D10598F0C6010E941E4DC70155E055
:109AF000969587955A95E1F70E94434D80E290E054
:109B0000E80EF91EC80ED91EA0970BC087010F5F83
:109B10001F4FC701F60161916F010E94CB4C219745
:109B200078012097C1F6DF91CF911F910F91FF909F
:109B3000EF90DF90CF900895DF93CF930F92CDB742
:109B4000DEB789830E94184C898190E065E0880F18
:109B5000991F6A95E1F7E0ECF1E01282918380832E
:109B600084E390E00E941D4C0F90CF91DF91089507
:109B7000EF92FF921F93DF93CF930F92CDB7DEB793
:109B800070ECE72E71E0F72E1091CA0189830E94D4
:109B9000BE4C0E94184C93E3D7011A969C931A97D7
:109BA00012961C92129711961C92119790E0E0EC7D
:109BB000F1E089819093C00184839F5F9032D1F757
:109BC000E0ECF1E012870F90CF91DF911F91FF90B1
:109BD000EF900895DF93CF930F92CDB7DEB78983CF
:109BE0000E94184C898190E0E5E0880F991FEA9562
:109BF000E1F7E0ECF1E012829183808382E390E070
:109C00000E941D4C0F90CF91DF9108951F93182F44
:109C10008FEF0E94B84D812F0E94EA4D1F91089549
:109C20000E94184C80E390E00E941D4C08958FEF35
:109C30000E94B84D0E94104E0895DF92EF92FF925D
:109C40000F931F93CF93DF937B018C01C0ECD1E086
:109C5000DA848AE38A87E882BB27A12F902F8F2D91
:109C60008983780100271127EA822C83BB27A52F3F
:109C7000942F832F8D839A01442755272E838BECB5
:109C800091E061E00E948348DA86DF91CF911F91D5
:109C90000F91FF90EF90DF900895EF92FF920F9356
:109CA0001F93DF93CF9300D00F92CDB7DEB77A0129
:109CB000890169837A838B839C830E94184C698114
:109CC0007A818B81382F9C81292F862F972FA32F64
:109CD000B22F0DC00BB6ABBFFC0127910BBEF70135
:109CE00021937F010196A11DB11D01501040011566
:109CF000110581F72496CDBFDEBFCF91DF911F9173
:109D00000F91FF90EF900895EF92FF920F931F93A2
:109D1000CF93DF937A018901EB01D1700AC081E012
:109D2000BE010E948946F70181937F01219601506F
:109D300010400115110599F7DF91CF911F910F91F7
:109D4000FF90EF9008952F923F924F925F926F9203
:109D50007F928F929F92AF92BF92CF92DF92EF92BB
:109D6000FF920F931F93DF93CF930F920F92CDB774
:109D7000DEB74A017901702E6B0166242E0108942A
:109D8000411C511C22242A94322C53C0A12C91E056
:109D9000B92E00E010E07720A9F081E0B8010E9420
:109DA0008946F2018083B8016F5F7F4F81E00E9496
:109DB0008946F201818389819A81FFEF8F3F9F0756
:109DC00021F405C029823A8202C066246394E1141A
:109DD000F104F9F0C016D10669F40894E108F1081D
:109DE0000894C11CD11CF40181914F018983E114B5
:109DF000F10479F0C8010196C816D90651F4089407
:109E0000E108F1080894C11CD11CF40181914F01B3
:109E10008A83B80180E090E049815A810E948607D8
:109E20000E5F1F4F0894A108B108A114B10409F0F6
:109E3000B2CFE114F10409F0A9CF662041F00E94ED
:109E4000184C60E070E0CB0148E10E9477070E9467
:109E5000184C60E070E0CB014AE10E9477070F9058
:109E60000F90CF91DF911F910F91FF90EF90DF90B6
:109E7000CF90BF90AF909F908F907F906F905F90AA
:109E80004F903F902F9008952F923F924F925F9264
:109E90006F927F928F929F92AF92BF92CF92DF92FA
:109EA000EF92FF920F931F93DF93CF93CDB7DEB75F
:109EB0002897CDBFDEBF1A0149010F83412C2EEF39
:109EC000522E2FEF622E2FEF722E4622572268223B
:109ED00079225B016C017DC00E94184CD301C20144
:109EE00080509E4FAF4FBF4F8B839C83AD83BE830B
:109EF0008301720120E09F81992369F00BB60BBFAB
:109F0000F701879196910BBE89839A83AFEF8F3FBC
:109F10009A0731F406C0EFEFFFEFE983FA8301C03F
:109F200021E08114910451F1AE14BF04C006D106A2
:109F300079F40894810891080894A11CB11CC11CF3
:109F4000D11CD1018D911D01898381149104B1F03F
:109F5000D801C7010196A11DB11DA816B906CA06F0
:109F6000DB0661F40894810891080894A11CB11CD7
:109F7000C11CD11CF10181911F018A8349815A8141
:109F8000C801B70128870E94860782E090E0A0E020
:109F9000B0E0E80EF91E0A1F1B1F28858B819C81EB
:109FA000AD81BE81E816F9060A071B0709F0A3CFA9
:109FB000222331F00E94184CC301B20145E205C0D2
:109FC0000E94184CC301B20144E20E9477072701A6
:109FD00038018114910409F07FCF2896CDBFDEBFF0
:109FE000CF91DF911F910F91FF90EF90DF90CF9075
:109FF000BF90AF909F908F907F906F905F904F90A9
:10A000003F902F9008950F931F93DF93CF930F925C
:10A01000CDB7DEB789830E94184C00EC11E089812E
:10A02000F801808387E090E00E941D4CF801848154
:10A030000F90CF91DF911F910F910895629FD001F2
:10A04000739FF001829FE00DF11D649FE00DF11DF3
:10A05000929FF00D839FF00D749FF00D659FF00DA2
:10A060009927729FB00DE11DF91F639FB00DE11D8F
:10A07000F91FBD01CF0111240895991B79E004C097
:10A08000991F961708F0961B881F7A95C9F7809537
:10A09000089597FB092E07260AD077FD04D049D0F2
:10A0A00006D000201AF4709561957F4F0895F6F759
:10A0B000909581959F4F0895A1E21A2EAA1BBB1B74
:10A0C000FD010DC0AA1FBB1FEE1FFF1FA217B30784
:10A0D000E407F50720F0A21BB30BE40BF50B661F9A
:10A0E000771F881F991F1A9469F76095709580955E
:10A0F00090959B01AC01BD01CF01089597FB092EFE
:10A1000005260ED057FD04D0D7DF0AD0001C38F446
:10A1100050954095309521953F4F4F4F5F4F089593
:10A12000F6F790958095709561957F4F8F4F9F4F73
:10A130000895AA1BBB1B51E107C0AA1FBB1FA6178E
:10A14000B70710F0A61BB70B881F991F5A95A9F7E0
:10A1500080959095BC01CD010895EF92FF920F93E9
:10A160001F93CF93DF93689F8001699F100D789FA5
:10A17000100D1124C8010E94D250E82EE7017E0183
:10A18000F92EE701209731F08E2D60E070E0A801F4
:10A190000E949254CE01DF91CF911F910F91FF90B9
:10A1A000EF900895CF93DF938230910510F482E011
:10A1B00090E0E091BF32F091C03240E050E020E00A
:10A1C00030E026C06081718168177907E0F0681778
:10A1D000790781F4828193812115310531F0D9010C
:10A1E00012968D939C9313972BC08093BF329093BC
:10A1F000C03226C04115510519F06417750718F4CF
:10A20000AB01E901DF019F0172816381E72FF62F26
:10A210003097C1F64115510501F1481B590B4430E7
:10A22000510580F412968D919C911397209719F007
:10A230008A839B8304C08093BF329093C032FD0118
:10A24000329646C0FD01E40FF51F81939193425071
:10A2500050404D935C9311973BC02091BD3230919B
:10A26000BE322115310541F420917D2F30917E2F92
:10A270002093BD323093BE3220917F2F3091802FBA
:10A280002115310541F42DB73EB740917B2F5091F8
:10A290007C2F241B350BE091BD32F091BE32E217CA
:10A2A000F307A0F42E1B3F0B2817390778F0AC01F9
:10A2B0004E5F5F4F2417350748F04E0F5F1F4093E6
:10A2C000BD325093BE328193919302C0E0E0F0E042
:10A2D000CF01DF91CF910895CF93DF93009709F4D9
:10A2E00091C0FC013297128213826091BF3270914B
:10A2F000C0326115710581F420813181280F391F29
:10A300008091BD329091BE328217930799F5E09308
:10A31000BD32F093BE3276C0DB0180E090E002C037
:10A32000CD01D901AE17BF0748F412962D913C918B
:10A33000139721153105A1F7CD0121C0A283B38365
:10A34000EF01499159919E01240F351FA217B307C0
:10A3500079F42D913C911197240F351F2E5F3F4FBB
:10A360002083318312962D913C911397228333835E
:10A37000009729F4E093BF32F093C03243C0DC0170
:10A380001296ED93FC9313974D915D91A40FB51F19
:10A39000EA17FB0769F420813181240F351F2E5FF6
:10A3A0003F4FEC0128833983228133812A833B8309
:10A3B000E0E0F0E002C0FB01BC01DB0112968D91F0
:10A3C0009C9113970097B9F79B012E5F3F4F8D919A
:10A3D0009C911197820F931F4091BD325091BE32D4
:10A3E0004817590779F4309729F41092BF32109228
:10A3F000C03202C012821382225030402093BD32FC
:10A400003093BE32DF91CF9108958F929F92AF9299
:10A41000BF92CF92DF92EF92FF920F931F93CF9351
:10A42000DF938C01CB010115110529F40E94D25054
:10A43000082F192FB5C0D80112979801260F371F82
:10A440002A173B0708F4AAC0ED90FC901197E61676
:10A45000F706D0F045E0E416F10408F4A1C0A70126
:10A46000445050404617570708F49AC0A70142507D
:10A470005040461B570BF901419351936D937C93C8
:10A48000CF010E946C518CC05B01AE18BF0848011F
:10A490008E0C9F1CE091BF32F091C032CC24DD24A1
:10A4A000C0E0D0E041C0E815F90599F560817181FF
:10A4B000AB014E5F5F4F4A155B0558F1AB014A197E
:10A4C0005B09CC24DD246894C1F8C40ED51E8280BB
:10A4D000A380E5E0CE16D10448F0F9018282A38280
:10A4E000408351838D939C93119709C0C7010296B5
:10A4F000860F971F8D939C931197E82DFA2D209727
:10A5000019F0EA83FB834CC0E093BF32F093C03272
:10A5100047C040815181C416D50608F46A01EF0195
:10A5200052814381E52FF42F309709F0BCCF409141
:10A53000BD325091BE3248155905E9F4C816D90606
:10A54000D0F440917F2F5091802F4115510541F457
:10A550004DB75EB760917B2F70917C2F461B570BD8
:10A5600024173507D8F42093BD323093BE328D9333
:10A570009C93119715C00E94D250C82EE6016E011F
:10A58000D92EE601209751F08C2DB801A7010E9429
:10A590007754C8010E946C51860102C000E010E0AF
:10A5A000C801DF91CF911F910F91FF90EF90DF9045
:10A5B000CF90BF90AF909F908F9008952F923F9231
:10A5C0004F925F927F928F929F92AF92BF92CF9263
:10A5D000DF92EF92FF920F931F93CF93DF934B0184
:10A5E000EA016115710519F0FB01808391832097C1
:10A5F00039F09E01225030402332310508F0F4C07A
:10A60000A82EB92EF50111915F017F01812F90E0F5
:10A610000E9429540097B1F71D3229F4F5011191D8
:10A620007F0101E006C01B3219F4F50111917F0191
:10A6300000E0209719F0C031D105B9F4103381F44E
:10A64000F7018081883711F0883551F4F7011181C5
:10A6500082E090E0E80EF91E0260C0E1D0E005C0A3
:10A66000209719F41033C1F422C0C830D105F9F095
:10A67000C930D10524F4C230D10509F507C0CA306C
:10A68000D10551F0C031D105D1F427C0A12CB12C96
:10A69000C12CF0E4DF2E26C0CAE0D0E0ECECAE2EF8
:10A6A000ECECBE2EECECCE2EECE0DE2E1BC0C8E0B7
:10A6B000D0E0A12CB12CC12C70E1D72E13C09E018B
:10A6C000442737FD4095542F60E070E080E090E82B
:10A6D0000E945C5059016A0105C0A12CB12CC12C0B
:10A6E00068E0D62E40E060E070E0CB011E0144241B
:10A6F00037FC4094542C50ED752E710EE72DEA3046
:10A7000070F0212F21542A3118F439EC732E06C031
:10A71000212F21562A3130F529EA722E710E272D6C
:10A7200030E02C173D07F4F447FD18C0A616B70615
:10A73000C806D90680F0A20191010E941E50670D43
:10A74000711D811D911D6130F0E07F07F0E08F07E2
:10A75000F0E89F0710F04FEF01C041E0F7011191C1
:10A760007F01C9CF8114910491F0442339F00894FA
:10A77000E108F108F401E082F18209C001FF1BC089
:10A78000970122503040F4012083318314C047FFE9
:10A7900012C000FF05C060E070E080E090E804C0F7
:10A7A0006FEF7FEF8FEF9FE722E230E02093C1321F
:10A7B0003093C23216C000FF08C090958095709506
:10A7C00061957F4F8F4F9F4F0CC097FF0AC082E269
:10A7D00090E08093C1329093C2326FEF7FEF8FEFA2
:10A7E0009FE79B01AC0103C020E030E0A901B90163
:10A7F000CA01DF91CF911F910F91FF90EF90DF90F1
:10A80000CF90BF90AF909F908F907F905F904F9030
:10A810003F902F900895FC0188279927E894219173
:10A820002032E9F3293010F02E30C8F32B3241F0FA
:10A830002D3239F4689404C00E940955820F911D8D
:10A84000219120532A30C0F31EF4909581959F4F9B
:10A85000089591114FC6803219F089508550D0F774
:10A860000895FB01DC0102C005900D92415050405B
:10A87000D8F70895FC0105900020E9F780959095A0
:10A880008E0F9F1F0895EF92FF920F931F93DF93F8
:10A89000CF930F920F92CDB7DEB7BC01DC010D90C4
:10A8A0000020E9F7CD01861B970B69837A830E940C
:10A8B000D2508C0169817A81009711F00E94C054B6
:10A8C000C8010F900F90CF91DF911F910F91FF90D2
:10A8D000EF900895FB01DC0104C08D910190801977
:10A8E00021F441505040C8F7881B990B0895FB0193
:10A8F000DC0102C001900D9241505040D8F70895FC
:10A900006817790768F4FB01DC01E40FF51FA40F59
:10A91000B51F02C002900E9241505040D8F70895E2
:10A920000C947754DC0101C06D9341505040E0F726
:10A930000895FB01DC018D9181341CF08B350CF402
:10A94000805E619161341CF06B350CF4605E861B97
:10A95000611189F3990B0895FC018191861721F00B
:10A960008823D9F7992708953197CF010895FB01DE
:10A97000DC018D91019080190110D9F3990B089594
:10A98000FB01DC0101900D920020E1F70895FB012D
:10A99000DC014150504030F08D910190801919F444
:10A9A0000020B9F7881B990B0895FB01DC01415089
:10A9B000504048F001900D920020C9F701C01D924F
:10A9C00041505040E0F70895FC0181E090E0019093
:10A9D000061609F4CF010020D1F701970895FB0175
:10A9E00051915523A9F0BF01DC014D91451741114B
:10A9F000E1F759F4CD010190002049F04D91401547
:10AA00004111C9F3FB014111EFCF81E090E00197C3
:10AA100008957AE0979F902D879F802D910D1124A6
:10AA200008950F931F93DF93CF93CDB7DEB72E9783
:10AA3000CDBFDEBF0E891F89888D998D26E02C83BE
:10AA400009831A8397FF02C080E090E801978D8305
:10AA50009E839E01245E3F4FCE0101966A8D7B8DC1
:10AA6000A9010E9498554D815E8157FD0AC02F8132
:10AA70003885421753070CF49A01020F131FF8018F
:10AA800010822E96CDBFDEBFCF91DF911F910F9127
:10AA90000895DF93CF93CDB7DEB72E97CDBFDEBF3E
:10AAA00085E08C838C899D8989839A839E01285EA9
:10AAB0003F4FCE0101966E897F89A9010E945359AB
:10AAC0002E96CDBFDEBFCF91DF9108950F931F93D8
:10AAD000DF93CF93CDB7DEB72E97CDBFDEBF8C010E
:10AAE000CB01BA0146E04C8309831A8397FF02C069
:10AAF00080E090E801978D839E83CE010196A901A5
:10AB00000E9498554D815E8157FD0AC02F8138857E
:10AB1000421753070CF49A01020F131FF801108219
:10AB20002E96CDBFDEBFCF91DF911F910F9108957B
:10AB30002F923F924F925F926F927F928F929F924D
:10AB4000AF92BF92CF92DF92EF92FF920F931F933B
:10AB5000DF93CF93CDB7DEB72C97CDBFDEBF6C01AF
:10AB60001B018A01FC0116821782838181FFD1C1FA
:10AB70002E010894411C511CF6019381F10193FDB3
:10AB8000859193FF81911F01882309F4BEC185320D
:10AB900039F493FD859193FF81911F01853229F44A
:10ABA00090E0B6010E94E05AE7CFEE24FF2420E0B7
:10ABB0002032B0F48B3269F08C3228F4803251F0BC
:10ABC000833271F40BC08D3239F0803349F4216047
:10ABD0002CC02260246029C0286027C0206125C0C5
:10ABE00027FD2CC0382F30533A3098F426FF08C088
:10ABF0008E2D880FE82EEE0CEE0CE80EE30E15C03D
:10AC00008F2D880FF82EFF0CFF0CF80EF30E20622C
:10AC10000CC08E3221F426FD78C1206406C08C362B
:10AC200011F4206802C0883649F4F10193FD859142
:10AC300093FF81911F01882309F0BACF982F955473
:10AC4000933018F09052933028F40C5F1F4FFFE3BD
:10AC5000F9830DC0833631F0833771F0833509F005
:10AC600060C022C0F801808189830E5F1F4F4201BE
:10AC700071E0A72EB12C16C062E0662E712C600E1A
:10AC8000711EF8018080918026FF03C06E2D70E058
:10AC900002C06FEF7FEFC4012C870E94935A5C01C2
:10ACA00083012C852F7717C052E0652E712C600E22
:10ACB000711EF8018080918026FF03C06E2D70E028
:10ACC00002C06FEF7FEFC4012C870E94885A5C019D
:10ACD0002C852068830123FD20C008C080E290E01D
:10ACE000B6012C870E94E05AFA942C858F2D90E0B3
:10ACF000A816B90698F311C0F40127FD859127FF26
:10AD000081914F0190E0B6012C870E94E05A2C857A
:10AD1000F110FA940894A108B108A114B10461F7E4
:10AD2000F1C0843611F0893649F527FF08C0F801D3
:10AD300060817181828193810C5F1F4F09C0F8018E
:10AD400060817181882777FD8095982F0E5F1F4F56
:10AD50004FE6B42EB22297FF09C09095809570956A
:10AD600061957F4F8F4F9F4FF0E8BF2AA2012AE0E5
:10AD700030E00E94275B782E741845C0853731F487
:10AD80003FEEB32EB2222AE030E025C099EFB92E73
:10AD9000B2228F36C1F0803720F4883509F0B5C073
:10ADA0000DC0803721F0883709F0AFC002C020E124
:10ADB000B22AB4FE0BC084E0B82A08C0B4FE09C0B1
:10ADC000E6E0BE2A06C028E030E005C020E130E021
:10ADD00002C020E132E0B7FE08C0F8016081718155
:10ADE000828193810C5F1F4F07C0F80160817181E0
:10ADF00080E090E00E5F1F4FA2010E94275B782E3B
:10AE00007418FFE7BF22B6FE0BC02EEFB2227E14ED
:10AE100038F4B4FE07C0B2FC05C08FEEB82202C001
:10AE2000A72C01C0AE2C8B2D90E0B4FE0DC0FE010E
:10AE3000E70DF11D2081203319F4E9EEBE2209C08F
:10AE4000A394B2FE06C004C086789070009709F003
:10AE5000A3948B2C9924B3FC14C0B0FE0FC0AF1484
:10AE600028F4E72CEF0CEA18AF2C08C0E72C06C03A
:10AE700080E290E0B6010E94E05AA394AF14C0F3C0
:10AE800004C0AF1410F4FA1801C0FF2484FE0FC0F0
:10AE900080E390E0B6010E94E05A82FE1FC081FE6E
:10AEA00003C088E590E010C088E790E00DC0C401C1
:10AEB00086789070009791F081FC02C080E201C01A
:10AEC0008BE2B7FC8DE290E0B6010E94E05A06C02A
:10AED00080E390E0B6010E94E05AEA947E14C0F349
:10AEE0007A94F201E70DF11D808190E0B6010E9495
:10AEF000E05A7720A9F706C080E290E0B6010E94F0
:10AF0000E05AFA94FF20C1F737CEF6012681378147
:10AF100002C02FEF3FEFC9012C96CDBFDEBFCF910E
:10AF2000DF911F910F91FF90EF90DF90CF90BF9036
:10AF3000AF909F908F907F906F905F904F903F90D9
:10AF40002F90089520FD09C0FC0123FD05C022FFBC
:10AF500002C073836283518340830895EF92FF920E
:10AF60000F931F9344FD10C046FD10C0DB01FC0190
:10AF7000AA0FBB1FEE1FFF1F1094D1F76A0F7B1F94
:10AF80008E1F9F1F31E003C033E001C034E0660F25
:10AF9000771F881F991F3150D1F77B018C01E20E7A
:10AFA000F11C011D111DA8019701B701CA011F91D4
:10AFB0000F91FF90EF900895EF92FF920F931F93E0
:10AFC000CF93DF938C01C8010E949E5AEC0197FD3C
:10AFD00008C00E9429540097B1F7CE01B8010E9421
:10AFE0000C5BCE01DF91CF911F910F91FF90EF90FD
:10AFF00008958F929F92AF92BF92DF92EF92FF924D
:10B000000F931F93DF93CF930F92CDB7DEB74C0111
:10B01000D62E5A01122F0E949E5A8B3219F08D3271
:10B0200049F41068DA9409F46CC0C4010E949E5A75
:10B0300097FD67C0312F3D7F232F2073F1F48033BC
:10B04000E1F4DA9409F448C0C40139830E949E5A9D
:10B05000398197FD41C03260883711F0883559F445
:10B060003064DA94C9F1C40139830E949E5A39814F
:10B0700097FF03C031C036FF3061EE24FF24870103
:10B08000282F2053283090F034FD09C02A3070F06A
:10B0900036FF05C02F7D422F4151463030F0B401BC
:10B0A00039830E940C5B398114C02750C801B70155
:10B0B000432F39830E94AE577B018C013981326066
:10B0C000DA9469F0C40139830E949E5A398197FF4E
:10B0D000D7CF31FD04C015C0EE24FF24870137FF10
:10B0E00008C010950095F094E094E11CF11C011D3E
:10B0F000111DC501B801A701232F0E94A25781E0AD
:10B1000001C080E00F90CF91DF911F910F91FF90D0
:10B11000EF90DF90BF90AF909F908F9008956F92C7
:10B120007F928F929F92AF92BF92CF92DF92EF92D7
:10B13000FF920F931F93DF93CF93CDB7DEB7A19705
:10B14000CDBFDEBF6C018A0179019E012F5F3F4FA9
:10B1500080E2F90111928A95E9F7F601838080E097
:10B1600090E0BB24992470E0A1E0B0E0F70183FCFB
:10B17000A59083FEA1907F01AA2009F47FC0FA2D3B
:10B18000FE3511F4009751F1472F50E04817590749
:10B1900044F44A2D4D3551F14D3219F4992001F105
:10B1A00003C0992009F4BA2C4A2D46954695469538
:10B1B000F901E40FF11D4A2D47703D0102C0660CF4
:10B1C000771C4A95E2F7908096289082AB1459F04C
:10B1D000AB1410F4A394E8CFAA94E6CF71E004C0B6
:10B1E0009924939401C099240196C0CF992019F015
:10B1F0008E8180628E83772351F0CE018196FE018D
:10B200003196208120952193E817F907D1F7BB24C7
:10B21000B3944E010894811C911C01C0BB24C6014B
:10B2200069A30E949E5A69A197FD20C0282F2695E8
:10B2300026952695F401E20FF11D208130E0AC0146
:10B240004770507002C0359527954A95E2F720FD6A
:10B2500004C0B6010E940C5B09C00115110519F06C
:10B26000F80181938F016150C9F602C0BB2031F40F
:10B270000115110529F0F801108202C0EE24FF2407
:10B28000C701A196CDBFDEBFCF91DF911F910F9176
:10B29000FF90EF90DF90CF90BF90AF909F908F90F6
:10B2A0007F906F9008954F925F926F927F929F92DE
:10B2B000AF92BF92CF92DF92EF92FF920F931F93C4
:10B2C000DF93CF930F92CDB7DEB77C016B013A01CC
:10B2D000FC011682178200E0E9C0812F90E00E94F5
:10B2E0002954009721F0C7010E94DC57DFC01532B6
:10B2F00041F4F601A3FC3591A3FE31916F01353283
:10B3000061F4C7010E949E5A97FDDCC0181709F42A
:10B31000CDC0B7010E940C5BD7C03A3239F4A3FC10
:10B320003591A3FE31916F0111E001C010E0992425
:10B330000FC01260692D70E080E090E040E20E9452
:10B34000AE57962EF601A3FC3591A3FE31916F0105
:10B35000232F20532A3068F311FF03C0992019F4DA
:10B36000B3C099249A94383619F03C3689F409C050
:10B37000F601A3FC3591A3FE31916F01383641F4FB
:10B3800018601460F601A3FC3591A3FE31916F01A2
:10B39000332309F499C084E99EE0632F70E0398378
:10B3A0000E947D5A3981009709F48EC0812F10FDCB
:10B3B00008C0F3014080518042E050E0640E751EE9
:10B3C00002C0442455243E3651F4F701468157818A
:10B3D00060E070E0C201212F0E94A25767C033369F
:10B3E00091F481FD02C099249394C7010E949E5A52
:10B3F00097FD68C04114510419F0F20181932F01A7
:10B400009A9499F751C03B3559F4C701692DA201AF
:10B4100096010E948F586C01009709F045C03FC00B
:10B42000C70139830E94DC57398197FD4BC03F36F5
:10B4300059F1303728F4343629F1393639F527C037
:10B44000333719F0353711F51DC0C7010E949E5AD8
:10B450005C0197FD11C00E942954009729F0C50195
:10B46000B7010E940C5B08C04114510419F0F201AD
:10B47000A1922F019A9449F741145104A9F0F201C5
:10B48000108212C0106203C0106101C01064C701B5
:10B49000692DA201212F0E94F957882329F4F70171
:10B4A0008381807379F410C010FF0F5FF701A380D0
:10B4B000F601A3FC1591A3FE11916F01112309F070
:10B4C0000CCF02C0002311F010E002C00FEF1FEFFD
:10B4D000C8010F90CF91DF911F910F91FF90EF90D6
:10B4E000DF90CF90BF90AF909F907F906F905F90D4
:10B4F0004F900895992788270895FC010590061616
:10B5000021F00020D9F7C00108953197CF010895A7
:10B51000FC010590615070400110D8F7809590951E
:10B520008E0F9F1F0895FC01615070400190011023
:10B53000D8F7809590958E0F9F1F0895CF93DF9336
:10B54000EC013B8130FF36C036FF09C03F7B3B83B7
:10B550008E819F8101968E839F832A8129C032FF2D
:10B560000FC0E881F9818081992787FD9095009728
:10B5700019F430623B831EC03196E883F98311C011
:10B58000EA85FB85CE01199597FF0BC02B813FEF14
:10B590008F3F930711F480E101C080E2822B8B83FF
:10B5A00009C02E813F812F5F3F4F2E833F83282F7D
:10B5B00030E002C02FEF3FEFC901DF91CF91089536
:10B5C0000F931F93CF93DF938C01EB018B8181FF4E
:10B5D0001BC082FF0DC02E813F818C819D81281769
:10B5E000390764F4E881F9810193E883F98306C09F
:10B5F000E885F985802F1995009731F48E819F8118
:10B6000001968E839F8302C00FEF1FEFC801DF9169
:10B61000CF911F910F910895FB01238120FF13C04B
:10B6200026FD11C03FEF8F3F930769F082832064AE
:10B630002F7D238326813781215030402683378315
:10B64000282F30E002C02FEF3FEFC9010895FA0123
:10B65000AA27283051F1203181F1E8946F936E7F51
:10B660006E5F7F4F8F4F9F4FAF4FB1E03ED0B4E042
:10B670003CD0670F781F891F9A1FA11D680F791F83
:10B680008A1F911DA11D6A0F711D811D911DA11D94
:10B6900020D009F468943F912AE0269F11243019A4
:10B6A000305D3193DEF6CF010895462F4770405D3F
:10B6B0004193B3E00FD0C9F7F6CF462F4F70405DEE
:10B6C0004A3318F0495D31FD4052419302D0A9F749
:10B6D000EACFB4E0A6959795879577956795BA9543
:10B6E000C9F700976105710508959B01AC010A2E09
:10B6F00006945795479537952795BA95C9F7620FE0
:0EB70000731F841F951FA01D0895F894FFCF9E
:10B70E00200000252D3230732025730A0D0025737D
:10B71E00202D2068657864756D70286C656E3D25EA
:10B72E0064293A0A0D002530347820200025303265
:10B73E00782000202020003A200020202025730AA7
:10B74E000D00082008000A0D00636F6D6D616E64B8
:10B75E00206E6F7420666F756E643A25730A0D0045
:10B76E0025732000256300240068656C70007072DC
:10B77E00696E74207468697320696E666F726D618C
:10B78E0074696F6E002573202D2068657864756D61
:10B79E0070286C656E3D2564293A0A0D00253034FB
:10B7AE0078202000253032782000202020003A20FA
:10B7BE000020202025730A0D007375636365737373
:10B7CE0000756E6B6E6F776E00616C726561647979
:10B7DE0020696E207573650061626F727465640016
:10B7EE0073796E63206572726F720063616E63654A
:10B7FE006C65642062792072656D6F74650069678F
:10B80E006E6F7265640074696D656F757400707229
:10B81E006F746F636F6C206572726F720064697300
:10B82E0061626C6564006275737900726574727919
:10B83E00206C61746572006261642073697A6500C0
:10B84E006F7574206F662072616E6765006F70652C
:10B85E00726174696F6E206E6F7420737570706F85
:10B86E0072746564006E6F207065726D69737369B2
:10B87E006F6E00696E636F6D70617469626C6520C6
:10B88E00747970650070617468206E6F7420666FD5
:10B89E00756E640070617273696E67206572726F87
:10B8AE007200696E76616C696420737461746500F0
:10B8BE006E6F7420636F6E6E6563746564006F7572
:10B8CE0074206F66206D656D6F72792F6275666676
:10B8DE0065727300696E76616C6964207061726165
:10B8EE006D657465727300756E6B6E6F776E206624
:10B8FE0061696C7572650073772076657273696F16
:10B90E006E3A25642E25642E25640A0D00636F6E33
:10B91E006E5F636220736F636B69643A25642063A4
:10B92E006F6E6E65637465643A25640A0D006F6B05
:10B93E000065727200257320256420282573290A5C
:10B94E000D0075736167653A207365745F706F6C77
:10B95E006C5F706572696F64203C706572696F64AC
:10B96E0020696E206D733E0A0D00706572696F64FA
:10B97E002025640A0D0075736167653A207365743E
:10B98E005F686561727462656174203C307C313E23
:10B99E000A0D0075736167653A207365745F6C6597
:10B9AE0064203C307C313E0A0D0000687474705F78
:10B9BE00706F7374004C697374656E696E67206F77
:10B9CE006E2025733A25642F25730A0D0075736159
:10B9DE0067653A2066775F75706772616465203CB3
:10B9EE006D6574686F642C20652E672E2022687436
:10B9FE0074705F706F7374223E205B3C69703E20E2
:10BA0E003C706F72743E203C706174683E5D0A0D2E
:10BA1E00006C6F6F6B75705F63623A20686F737442
:10BA2E00206E6F7420666F756E640A0D006C6F6FFA
:10BA3E006B75705F63622069703A25730A0D00257D
:10BA4E007320256420280069703A257320006D61EB
:10BA5E00736B3A2573200067773A25732000646E66
:10BA6E00733A2573290A0D00636170733A30782595
:10BA7E003032780A0D00756E6B6E6F776E006677DA
:10BA8E002076657273696F6E3A25642E25642E25B5
:10BA9E0064206275696C643A25730A0D006877201C
:10BAAE007265766973696F6E3A25730A0D00757348
:10BABE006167653A206765745F686F737462796E4B
:10BACE00616D65203C646E736E616D653E0A0D009E
:10BADE002573202564202825732920007065657242
:10BAEE003A25730A0D0075736167653A20676574B0
:10BAFE005F7065657261646472203C736F636B691D
:10BB0E00643E0A0D0073656E64696E6720256420BD
:10BB1E00627974657320746F2025733A25640A0D5B
:10BB2E000077726F74653A25642072656D61696E77
:10BB3E003A25640A0D0075736167653A2073656E68
:10BB4E0064746F203C736F636B69643E203C697054
:10BB5E003E203C706F72743E203C64617461202EF6
:10BB6E002E2E3E0A0D0073656E64696E6720256485
:10BB7E002062797465730A0D0075736167653A20EA
:10BB8E0073656E64203C736F636B69643E203C6426
:10BB9E00617461202E2E2E3E0A0D0075736167654D
:10BBAE003A20636C6F7365203C736F636B69643E00
:10BBBE000A0D0075736167653A20636F6E6E65637B
:10BBCE0074203C736F636B69643E203C69703E2049
:10BBDE003C706F72743E0A0D0075736167653A2092
:10BBEE006C697374656E203C736F636B69643E2081
:10BBFE005B6261636B6C6F675D0A0D006C697374D9
:10BC0E00656E5F636220736F636B69643A25642CA3
:10BC1E0020616363657074696E67202E2E2E20007E
:10BC2E0028636F6E6E656374696F6E206C6F7374CC
:10BC3E002900726563765F636220736F636B69645C
:10BC4E003A2564206C656E3A25642025730A0D0032
:10BC5E0052580075736167653A2062696E64203CC4
:10BC6E00736F636B69643E203C69703E203C706F5D
:10BC7E0072743E0A0D0073747265616D00646772B2
:10BC8E00616D007261770075736167653A20736F3D
:10BC9E00636B6574203C73747265616D7C6467724E
:10BCAE00616D7C7261773E205B70726F746F636F33
:10BCBE006C5D0A0D0075736167653A207365745F7C
:10BCCE006468637064203C307C313E0A0D0025733D
:10BCDE002025642028656E61626C65643A256429AE
:10BCEE000A0D0075736167653A207365745F646849
:10BCFE006370203C307C313E0A0D007573616765C0
:10BD0E003A207365745F697061646472203C697077
:10BD1E003E205B6D61736B5D205B67775D205B64BE
:10BD2E006E735D0A0D004E2F410025732025642091
:10BD3E000028257320253032783A253032783A257E
:10BD4E003032783A253032783A253032783A25300A
:10BD5E00327820727373693A256420736E723A25B5
:10BD6E0064290A0D00257320256420282530327899
:10BD7E003A253032783A253032783A253032783AD0
:10BD8E00253032783A25303278290A0D00757361E4
:10BD9E0067653A207365745F6368616E6E656C20CB
:10BDAE003C6368616E6E656C3E0A0D00582025641A
:10BDBE002025642025642025642025640075736188
:10BDCE0067653A20636F6E665F7073203C757365AE
:10BDDE005F70735F706F6C6C3E203C70735F74723B
:10BDEE0061666669635F74696D656F75743E0A0D91
:10BDFE000020202020202020202020202020202055
:10BE0E003C70735F64656C61793E203C72785F6153
:10BE1E006C6C5F6474696D3E203C6C697374656E06
:10BE2E005F696E74657276616C3E0A0D00757361A2
:10BE3E0067653A207365745F7073203C307C313EC9
:10BE4E000A0D007374610061700075736167653A65
:10BE5E00207365745F6D6F6465203C7374617C61E3
:10BE6E00703E0A0D00777061320077706100776561
:10BE7E00700075736167653A206C696E6B75702022
:10BE8E005B737369645D205B6B65795D205B7765C1
:10BE9E00707C7770617C777061325D0A0D0075730E
:10BEAE006167653A207365745F626175647261746F
:10BEBE0065203C62617564726174653E205B7274CC
:10BECE00736374735D0A0D006572722025642028F9
:10BEDE006661696C656420746F20636F6E66696756
:10BEEE0075726520686F73742075617274290A0DFE
:10BEFE0000726573657400776C705F72657365743C
:10BF0E002829007365745F626175647261746500DF
:10BF1E00776C705F7365745F62617564726174656E
:10BF2E002829006C696E6B757000776C705F6C6998
:10BF3E006E6B757028737369642C206B65792C2079
:10BF4E006175746829006C696E6B646F776E00772B
:10BF5E006C705F6C696E6B646F776E282900736509
:10BF6E00745F6D6F646500776C705F7365745F6D81
:10BF7E006F64652829006765745F6D6F646500776F
:10BF8E006C705F6765745F6D6F64652829007365FB
:10BF9E00745F707300776C705F7365745F70732875
:10BFAE002900636F6E665F707300776C705F636FEE
:10BFBE006E665F70732829007365745F6368616EC7
:10BFCE006E656C00776C705F7365745F6368616E2D
:10BFDE006E656C2829006765745F687761646472AA
:10BFEE0000776C705F6765745F6877616464722850
:10BFFE0029006765745F6E6574776F726B00776C7E
:10C00E00705F6765745F6E6574776F726B28290059
:10C01E007365745F69706164647200776C705F73CE
:10C02E0065745F6970616464722869702C206D613B
:10C03E00736B2C2067772C20646E732900676574F0
:10C04E005F69706164647200776C705F6765745FBE
:10C05E006970616464722829007365745F64686333
:10C06E007000776C705F7365745F646863702865C9
:10C07E006E61626C6529006765745F646863700049
:10C08E00776C705F6765745F6468637028290073EE
:10C09E0065745F646863706400776C705F73657459
:10C0AE005F6468637064282900736F636B65740046
:10C0BE00776C705F736F636B657428747970652C21
:10C0CE002070726F746F290062696E6400776C70F5
:10C0DE005F62696E6428736F636B2C2069702C200D
:10C0EE00706F727429006C697374656E00776C7072
:10C0FE005F6C697374656E28736F636B69642C2053
:10C10E006261636B6C6F672900636F6E6E6563743B
:10C11E0000776C705F636F6E6E65637428736F6308
:10C12E006B69642C2069702C20706F727429006307
:10C13E006C6F736500776C705F636C6F73652873DB
:10C14E006F636B6964290073656E6400776C705F52
:10C15E0073656E6428736F636B69642C20646174FD
:10C16E0061290073656E64746F00776C705F736520
:10C17E006E64746F28736F636B69642C20646174D2
:10C18E00612C2069702C20706F72742900676574A1
:10C19E005F706565726164647200776C705F67656D
:10C1AE00745F706565726164647228736F636B6926
:10C1BE006429006765745F686F737462796E616D70
:10C1CE006500776C705F6765745F686F7374627912
:10C1DE006E616D6528646E736E616D6529006765AD
:10C1EE00745F76657273696F6E007072696E74201B
:10C1FE00636C69656E742076657273696F6E006725
:10C20E0065745F66775F76657273696F6E007072C4
:10C21E00696E74206669726D7761726520766572DB
:10C22E0073696F6E006765745F66775F63617073C5
:10C23E00007072696E74206669726D776172652026
:10C24E006361706162696C69746965730066775FBA
:10C25E007570677261646500776C705F66775F7585
:10C26E00706772616465286D6574686F642C2061F7
:10C27E006464722C20706F72742C20706174682943
:10C28E00007365745F6C656400776C705F736574C2
:10C29E005F6C65642829007365745F6865617274EC
:10C2AE006265617400776C705F7365745F68656159
:10C2BE007274626561742829007365745F706F6CA7
:10C2CE006C5F706572696F6400776C705F73657414
:10C2DE005F706F6C6C5F706572696F642829000DFA
:10C2EE000A0047455420002D2D2D202573207069FE
:10C2FE006E672073746174697374696373202D2D76
:10C30E002D0A0D002564207061636B6574732074B3
:10C31E0072616E736D69747465642C20256420726D
:10C32E00656365697665640A0D002564206279741B
:10C33E0065732066726F6D2025733A2069636D7088
:10C34E005F7365713D25640A0D0025642062797462
:10C35E0065732066726F6D2025733A2069636D7068
:10C36E005F7365713D25642044657374696E6174F5
:10C37E00696F6E20486F737420556E7265616368C5
:10C38E0061626C650A0D0025642062797465732004
:10C39E0066726F6D2025733A2069636D705F7365E9
:10C3AE00713D256420547970653A25640A0D006F3D
:10C3BE006B00657272002D63002D730025732025AE
:10C3CE006420282573290A0D0075736167653A206C
:10C3DE0070696E67205B2D63203C636F756E743ED3
:10C3EE005D205B2D73203C73697A653E5D203C6950
:10C3FE00703E0A0D0070696E67000A0D007474635A
:10C40E0070206572723A256420282573290A0D0062
:10C41E0074746370206F6B3A2025642062797465A2
:10C42E00732070726F63657373656420696E202567
:10C43E006C75206D732C20256C75204B422F730A62
:10C44E000D0074746370206F6B3A2025642062793E
:10C45E007465732070726F63657373656420696EA3
:10C46E002030206D730A0D002E002D70002D6E00F1
:10C47E002D6C002D74002D7200257320256420284C
:10C48E002573290A0D00657272007474637020633F
:10C49E006F6E6E6563742025733A2564206E627527
:10C4AE00663A2564206275666C656E3A2564207363
:10C4BE006F636B69643A25640A0D007474637020AF
:10C4CE006C697374656E20706F72743A25642062A5
:10C4DE0075666C656E3A2564206C736F636B696468
:10C4EE003A25640A0D0075736167653A20747463AA
:10C4FE0070205B2D7472706E6C5D0A0D0074746327
:10C50E00700074746370207468726F7567687075EC
:10C51E00742074657374006661696C656420746F51
:10C52E0020676574206E74702074696D653A25738A
:10C53E00282564290A0D006E74702074696D653AA1
:10C54E0020253034642D253032642D253032642080
:10C55E00253032643A253032643A253032640A0D81
:10C56E00006F6B00657272002573202564202825EC
:10C57E0073290A0D0075736167653A206E74702019
:10C58E003C6E74702D7365727665723E0A0D006E88
:10C59E0074700067657420736572766572207469B5
:10C5AE006D652066726F6D206E7470004E2F4100A7
:10C5BE00253032783A253032783A253032783A259D
:10C5CE003032783A253032783A25303278002F00E2
:10C5DE002F3F002F696E6465782E68746D6C3F0076
:10C5EE00746F67676C653D4C45442564002F696E1A
:10C5FE006465782E68746D6C002F6C6F676F2E6794
:10C60E006966006C696E6B5F6362206C696E6B3A73
:10C61E0025640A0D00616464725F63622069703A7A
:10C62E006E6F6E650A0D0068747470642073746F9B
:10C63E00707065640A0D00616464725F63622069E4
:10C64E00703A25730A0D00687474706420737461F7
:10C65E00727465640A0D006864776972656C65733F
:10C66E0073006864776972656C6573733132330079
:10C67E00004E0045004F004D0053002000C3320015
:10C68E00006920D8176E2000000000F1273432F721
:10C69E002700000000032867311028000000002347
:10C6AE002892302A2800000000462856304F2800D5
:10C6BE000000005E28EA2F6728000000007628A8F8
:10C6CE002F7F28000000008E283C2F9528000000A8
:10C6DE0000A2284C2EAA2800000000B828E12DC484
:10C6EE002800000000D628942DE12800000000F25A
:10C6FE0028BE2CFE28000000001029FE2B1B29004E
:10C70E000000003D29BB2248290000000059299253
:10C71E002B6229000000007729542B80290000008D
:10C72E00008F29E82A992900000000A929372AB08C
:10C73E002900000000C829A929CD2900000000E623
:10C74E00295228ED2900000000092AC427112A00C9
:10C75E000000002F2A5827352A00000000472A75AE
:10C76E00264C2A00000000632A5F256A2A0000007A
:10C77E00008D2AD1249A2A00000000B32A7524C203
:10C78E002A00000000DE2A5B1FEA2A00000000FFDC
:10C79E002AD4230E2B00000000252B7423312B00EE
:10C7AE000000004D2B9521582B00000000812B29F5
:10C7BE0021892B00000000972B9820A52B0000004C
:10C7CE0000B92BD01FC92B00000000F52CE835F561
:10C7DE002C00000000FD2DBB39022E000000008F42
:10C7EE002E5B3C932E0000000000000000FFFFFFB8
:10C7FE00FFC920D820E020EB20FE2006210E211DAF
:10C80E002126212B21372140214D216521732185A0
:10C81E00219421A221B021BE21D421E72100001FA5
:10C82E00003B005A0078009700B500D400F30011C9
:10C83E000130014E016D0100001F003C005B0079CC
:10C84E00009800B600D500F400120131014F016EC0
:10C85E00010001020307712F732F752F772F792F88
:00000001FF
